:030000000272B0D9
:1072B00074FEF595F5B1F5B2F5B3F5B4F5E1745595
:0E72C000F5AE78FFE4F6D8FD75812302730960
:10633C002573004844575220202056455253494F4C
:10634C004E3A202020202573005346545752205695
:10635C00455253494F4E3A20202020257300414985
:10636C0053472020202056455253494F4E3A202067
:10637C002020322E30004149534720202020564502
:10638C005253494F4E3A20202020312E3100534594
:10639C00545550204D454E550041495347205645C4
:1063AC005253494F4E3A202575005343414E2054C9
:1063BC005950453A2048444C4320005343414E2009
:1063CC00545950453A20554E4951554520494400A1
:1063DC0000534156494E47204348414E47455300D0
:1063EC00505553482046494E4420544F204F504559
:1063FC0052415445005245414420444F574E544954
:10640C004C543A20252B23352E316600534554200D
:10641C00444F574E54494C542020203A20252B23CE
:10642C00352E3166005343414E3A202575005052AB
:10643C0045535320494E432F44454320544F20008D
:10644C004348414E4745204E4F2E204F462044494D
:10645C004749545320544F005052455353204649FA
:10646C004E4420544F20535441525400257500344F
:10647C002E3035003039435458445F534F465457EF
:03648C0041524535
:103936004601825245565F45004201780000420129
:0D3946007A000342017C0000420180000075
:10431400D2B3D20BE4900564F09000F9F0907FE002
:1043240004F09000FA74FFF0A374FBF09000FAE03C
:10433400FEA3E0F5828E83E0FF90097CE4F0A3EF16
:10434400F09000FA74FFF0A374F9F09000FAE0FE24
:10435400A3E0F5828E83E0900B1FF0E4900B51F004
:1043640090097CE07004A3E06401600990097CE496
:10437400F0A37402F0900B1FE060037401F0126468
:104384008F127752127C2EE49005CFF01275B2E4AE
:10439400FFFE127BC890013B74FFF0A37463F0A38B
:1043A400743CF0A37401F0A37400F0A374DFF07BF9
:1043B400017A057969123EF690013B74FFF0A3740B
:1043C40063F0A3743FF0A37401F0A37401F0A37429
:1043D40082F07B017A057982123EF690013B74FFEC
:1043E400F0A37463F0A37455F0A374FFF0A3746492
:1043F400F0A3747BF07B017A05799B123EF6900959
:104404007CE07004A3E06402701790013B74FFF039
:10441400A37463F0A3746AF07B017A0579B4123E45
:10442400F690097CE07004A3E06401701790013BEE
:1044340074FFF0A37463F0A37482F07B017A0579AE
:10444400B4123EF6127D289000F77455F0E4900003
:10445400F6F09000F7E0FF9000F6E0C39F400302FF
:104464004674127B93200903024618E590547FFF9B
:10447400900176E4F0A3EFF0900176E07004A3E0FD
:10448400641870E19000FC04F0900176E07004A3DD
:10449400E0640270030245F0E590547FFF900176DA
:1044A400E4F0A3EFF090013B74FFF0A37463F0A376
:1044B400749AF07B017A057969123EF690013B7497
:1044C400FFF0A37463F0A374A5F090097CE0FFA34C
:1044D400E090013ECFF0A3EFF07B017A05798212E0
:1044E4003EF6900B1FE0701790013B74FFF0A3742D
:1044F40063F0A374B6F07B017A05799B123EF690C3
:104504000B1FE0B4011790013B74FFF0A37463F038
:10451400A374C7F07B017A05799B123EF690013BA8
:1045240074FFF0A37463F0A374DCF07B017A057963
:10453400B4123EF6E49000F8F09000F8E0FFC39463
:10454400045032E4900564F09000FCE0FEEFB50600
:10455400069005647401F09000F8E0FF75F019A46A
:104564002469F582E43405AD82FC125ADB9000F82C
:10457400E004F080C4900176E0FEA3E0FF64044E02
:1045840070069000FC7402F0EF64084E7005900011
:10459400FC04F0EF64204E703C9000F904F09000AD
:1045A400FCE0B4012390097DE004F0700690097CDE
:1045B400E004F090097CE07004A3E06403701690BA
:1045C400097CF0A304F0800D900B1FE06401F090CF
:1045D40000F97401F0900978E0FCA3E0FDA3E0FE8B
:1045E400A3E0FF12235812786D02448D9000F9E085
:1045F400B4011A90013B74FFF0A37463F0A374DD5B
:10460400F07B017A0579B4123EF6127D287F907E04
:104614000112786D9000F9E06401704B907FE00422
:10462400F09000FA74C0F0A3E4F0FF7EC01277B2F9
:104634009000FA74FFF0A374FBF090097CA3E0905F
:1046440000F8F0FD7FFB7EFF12753F9000FA74FFC7
:10465400F0A374F9F0900B1FE09000F8F0FD7FF9DF
:104664007EFF12753F80099000F6E004F002445684
:1046740090097CE0FEA3E0FF64014E7018900B5398
:1046840074FFF0A37472F0A37460F090154C74126C
:10469400F0A374E8F0EF64024E7018900B5374FFAB
:1046A400F0A37472F0A37410F090154C7412F0A37C
:1046B40074E7F090013B74FFF0A37463F0A3743CBF
:1046C400F0A37401F0A37400F0A374DFF07B017A0B
:1046D400057969123EF690013B74FFF0A37463F010
:1046E400A374DCF07B017A057982123EF690013BDB
:1046F40074FFF0A37463F0A374DCF07B017A057992
:104704009B123EF690013B74FFF0A37463F0A37414
:10471400ECF07B017A0579B4123EF6127D28E49020
:1047240005CDF0A3F0900567F0A3F0900986122957
:104734001F0000000090098212291F000000009051
:104744000B3612291F00000000E4900B50F0900B70
:0247540052F021
:014756002240
:107D5C00E590547F6401700DC20BC2C3C2B37FB8EF
:057D6C007E0B12786D92
:017D710022EF
:102ACD00E590547FFF90017EE4F0A3EFF0A3E0FECC
:102ADD00A3E0FF90017EE0FCA3E0FD6F7002EC6EC1
:102AED0070030232A1EC60030232A1ED70030232D9
:102AFD009424FE604424FE7003022D3424FC7003E4
:102B0D00022E9C24F8700302300B24F07003023166
:102B1D00B124E07003023236243F60030232A1205B
:102B2D000B07D20BD2B3023294C20BC2C3C2B37F16
:102B3D00B87E0B12786D023294900B3612291F005D
:102B4D00000000D2C3900567E07002A3E07003029D
:102B5D002D1F90017CE07002A3E06003022D1F90F9
:102B6D000B5104F0126CFF90017CEEF0A3EFF04ED0
:102B7D00600D126F6AE490017CF0A3F0022D1F909E
:102B8D000982E0FCA3E0FDA3E0FEA3E0FF900B783B
:102B9D00122913E49000F6F0A3F09000F7E004F092
:102BAD0070069000F6E004F0900982E0FCA3E0FDD1
:102BBD00A3E0FEA3E0FF900B78E0F8A3E0F9A3E01B
:102BCD00FAA3E0FB1222AD6007E49000F6F0A3F04B
:102BDD007FFA7E0012786D900982E0FCA3E0FDA3E0
:102BED00E0FEA3E0FF900B781229139005CFE0FFD4
:102BFD0012695090017CEEF0A3EFF04E703490010D
:102C0D003B74FFF0A37464F0A37401F0900982E0AB
:102C1D00FCA3E0FDA3E0FEA3E0FF90013E1229130B
:102C2D007B017A0579B4123EF67C057DB47F0312E3
:102C3D005ADB90017CE07002A3E0600A126F6AE437
:102C4D0090017CF0A3F0127D5CE4FFFE7D207C41C1
:102C5D00900986E0F8A3E0F9A3E0FAA3E0FB1221C6
:102C6D0007E4FBFA798078BF122016C004C005C0B6
:102C7D0006C007E4FFFE7D207C41900982E0F8A3A9
:102C8D00E0F9A3E0FAA3E0FB122107A804A905AA25
:102C9D0006AB07D007D006D005D0041222AD406098
:102CAD00E4FFFE7D207C41900986E0F8A3E0F9A3C6
:102CBD00E0FAA3E0FB122107E4FBFA7980783F12DA
:102CCD002016C004C005C006C007E4FFFE7D207CB1
:102CDD0041900982E0F8A3E0F9A3E0FAA3E0FB122A
:102CED002107A804A905AA06AB07D007D006D00571
:102CFD00D0041222AD60025007E4900B51F0801207
:102D0D00D39000F7E0940C9000F6E094005003028D
:102D1D002BA790017EE0FFA3E0A3CFF0A3EFF0E49B
:102D2D00900B51F00232A1900B3612291F000000BA
:102D3D0000D2C3900567E07002A3E07003022E2A53
:102D4D0090017CE07002A3E06003022E2AE590540E
:102D5D007F64046003022E2A9007D0E0FCA3E0FDFF
:102D6D00A3E0FEA3E0FF900986E0F8A3E0F9A3E05D
:102D7D00FAA3E0FB1222AD5003022E2A900986E041
:102D8D00FCA3E0FDA3E0FEA3E0FFE4FBFA7980786D
:102D9D00BE1220169009861229139007D0E0FCA3CD
:102DAD00E0FDA3E0FEA3E0FF900986E0F8A3E0F9C3
:102DBD00A3E0FAA3E0FB1222AD50149007D0E0FC83
:102DCD00A3E0FDA3E0FEA3E0FF9009861229139076
:102DDD00013B74FFF0A37464F0A37418F09009869E
:102DED00E0FCA3E0FDA3E0FEA3E0FF90013E12296D
:102DFD00137B017A05799B123EF67C057D9B7F0244
:102E0D00125ADB120007900978E0FCA3E0FDA3E065
:102E1D00FEA3E0FF12235812786D022D5A9001780F
:102E2D00E07004A3E064017063900567E07002A395
:102E3D00E0705990017CE07002A3E0704F90017B2F
:102E4D00E024FFF090017AE034FFF0C3A3E0940199
:102E5D0090017AE094005005E4F0A304F090013B5A
:102E6D0074FFF0A37464F0A37431F090017AE0FF65
:102E7D00A3E090013ECFF0A3EFF07B017A05799BA3
:102E8D00123EF67C057D9B7F02125ADB0232949036
:102E9D000B3612291F00000000D2C3900567E070A9
:102EAD0002A3E07003022F9690017CE07002A3E074
:102EBD006003022F96E590547F64086003022F96FD
:102ECD009007D4E0FCA3E0FDA3E0FEA3E0FF900992
:102EDD0086E0F8A3E0F9A3E0FAA3E0FB1222AD60CF
:102EED00054003022F96900986E0FCA3E0FDA3E0C8
:102EFD00FEA3E0FFE4FBFA7980783E1220169009DC
:102F0D00861229139007D4E0FCA3E0FDA3E0FEA3F5
:102F1D00E0FF900986E0F8A3E0F9A3E0FAA3E0FB57
:102F2D001222AD601640149007D4E0FCA3E0FDA37F
:102F3D00E0FEA3E0FF90098612291390013B74FF78
:102F4D00F0A37464F0A37418F0900986E0FCA3E07C
:102F5D00FDA3E0FEA3E0FF90013E1229137B017A51
:102F6D0005799B123EF67C057D9B7F02125ADB1282
:102F7D000007900978E0FCA3E0FDA3E0FEA3E0FFCD
:102F8D0012235812786D022EC2900178E07004A3BE
:102F9D00E064017066900567E07002A3E0705C90DC
:102FAD00017CE07002A3E0705290017BE004F070B0
:102FBD000690017AE004F0D390017BE09408900133
:102FCD007AE094004006E4F0A37408F090013B749D
:102FDD00FFF0A37464F0A37431F090017AE0FFA3C5
:102FED00E090013ECFF0A3EFF07B017A05799B12C3
:102FFD003EF67C057D9B7F02125ADB023294900BCC
:10300D003612291F00000000D2C3900178E0700431
:10301D00A3E06401600302311B900B50E0FFD394D9
:10302D000040279005CFE08FF084E5F004FFF0120B
:10303D0068417E0090017CEEF0A3EFF06026126FE8
:10304D006AE490017CF0A3F0801AE490017CF0A377
:10305D00F090017AE0FEA3E0FF123325900567EEB4
:10306D00F0A3EFF0900567E07002A3E0707190019E
:10307D0078F0A3F090013B74FFF0A37463F0A37498
:10308D003CF0A37401F0A37400F0A374DFF07B0196
:10309D007A057969123EF690013B74FFF0A37463D3
:1030AD00F0A374DCF07B017A057982123EF6900173
:1030BD003B74FFF0A37463F0A374DCF07B017A051D
:1030CD00799B123EF690013B74FFF0A37463F0A35D
:1030DD0074ECF07B017A0579B4123EF6127D2890DE
:1030ED000567E07002A3E0600B1258DF90017CEEE3
:1030FD00F0A3EFF090017CE07002A3E070030231C9
:10310D00AE126F6AE490017CF0A3F00231AE900133
:10311D007AE4F0A37403F0900B1FE0700790017A2E
:10312D00F0A304F0900178E4F0A304F0E49005CD51
:10313D00F0A3F090013B74FFF0A37464F0A3743A14
:10314D00F07B017A057969123EF690013B74FFF030
:10315D00A37464F0A3744CF07B017A057982123E5E
:10316D00F690013B74FFF0A37464F0A37431F090FA
:10317D00017AE0FFA3E090013ECFF0A3EFF07B01D9
:10318D007A05799B123EF690013B74FFF0A37464AF
:10319D00F0A37464F07B017A0579B4123EF6127DCA
:1031AD0028023294900B3612291F00000000D2C362
:1031BD00900567E07002A3E0606D90017CE0700205
:1031CD00A3E07063900B76E0FCA3E0FD900B7CE038
:1031DD00FEA3E0FF1226EBED2401FEE43C900B7CF8
:1031ED00F0A3CEF090013B74FFF0A37463F0A374D1
:1031FD003CF0900B7CE0FEA3E0FF7C007D191226D5
:10320D00D974C12FF974093EFA90013E7401F0A3EF
:10321D00EAF0A3E9F07B017A057982123EF67C058E
:10322D007D827F01125ADB805E900B3612291F00C2
:10323D00000000D2C3900567E07002A3E0604690E5
:10324D00017CE07002A3E0703C900B74E0FCA3E005
:10325D00FD900B3AE0FEA3E0FF1226EBED2401FFFB
:10326D00E43CFE900B3AF0A3EFF0127BC81258DF4E
:10327D0090017CEEF0A3EFF04E600A126F6AE490BD
:10328D00017CF0A3F0800090017EE0FFA3E0A3CFCE
:10329D00F0A3EFF0900B36E0FCA3E0FDA3E0FEA35E
:1032AD00E02401FFE43EFEE43DFDE43CFC900B36E2
:1032BD00122913E47B4A7A01F9F8900B6EE0FCA316
:1032CD00E0FDA3E0FEA3E0FF12284F900B36E0F8DF
:1032DD00A3E0F9A3E0FAA3E0FBD31228EF4002C26A
:1032ED00C3E47B32FAF9F8900B6EE0FCA3E0FDA38A
:1032FD00E0FEA3E0FF12284F900B36E0F8A3E0F9B3
:10330D00A3E0FAA3E0FBC31228EF400BC2C3C2B384
:07331D007FB87E0B12786DF2
:013324002286
:10734E00907FE07402F0906480E493FE740193FFEA
:10735E00908008E06E7003A3E06F600C900B6E12CD
:10736E00291F00B71B008014908000E0FCA3E0FDF5
:10737E00A3E0FEA3E0FF900B6E12291390013B7465
:10738E00FFF0A37464F0A37478F0908004E0FFA380
:10739E00E090013ECFF0A3EFF07B017A01798212EB
:1073AE003EF6E4907FE0F0D2C3127B24124314E445
:1073BE0090187DF012000712000312000790187D3E
:1073CE00E0B4010512601A8003122ACD1200078064
:0173DE00ECC2
:106CFF00E4901413F0A3F0D3900B75E09401900B74
:106D0F0074E09400403C900B3AA3E0FF90154CE0E8
:106D1F00FCA3E0F5828C83C083C082901413E475CA
:106D2F00F001122776FCD082D083E58225F0F58220
:106D3F00E5833CF583EFF09011B3E4F0A37481F099
:106D4F0080099011B3E4F0A37433F0E4FFFE7D20CB
:106D5F007C41900986E0F8A3E0F9A3E0FAA3E0FBF9
:106D6F00122107122358901543E4F0A37412F090E8
:106D7F00154CE0FAA3E0F5828A83C083C082901499
:106D8F0013E475F001122776FAD082D083E58225BD
:106D9F00F0F582E5833AF583EFF0EEFF90154CE0C6
:106DAF00FCA3E0F5828C83C083C082901413E4753A
:106DBF00F001122776FCD082D083E58225F0F58290
:0A6DCF00E5833CF583EFF012565007
:016DD9002297
:106950009011AFE4F0A3EFF0E4901413F0A3F0D3A0
:10696000900B75E09401900B74E09400403C900B08
:106970003AA3E0FF90154CE0FCA3E0F5828C83C0C5
:1069800083C082901413E475F001122776FCD08244
:10699000D083E58225F0F582E5833CF583EFF09026
:1069A00011B3E4F0A37482F080099011B3E4F0A372
:1069B0007434F0901543E4F0A37412F01256509022
:1069C00000FBEEF0A3EFF04E6002807DE490141126
:1069D000F0A3F0D3900B75E09401900B74E0940059
:1069E000400E901412E004F07006901411E004F0D0
:1069F000901412E02401FF901411E03400FE901571
:106A00004AE0FCA3E0FD2FF582EC3EF583E0FB7A43
:106A100000901412E02402FF901411E03400FEED07
:106A20002FF582EC3EF583E0FE7C00AD03E42BFF06
:106A3000EC3EFEAD07FC12231FE4FBFA79207841FF
:106A40001222109009821229139000FBE0FEA3E0AD
:016A5000FF46
:016A51002222
:106C21005343414E4E494E4720464F5220414E5408
:106C3100454E4E415300005343414E4E494E47206D
:106C41002020005343414E4E494E472020202575B8
:106C510000544845524520415245204D4F52452050
:106C61004445564943455300544F20424520464F21
:106C7100554E442E20494E435245415345005448F8
:106C810045204E554D424552204F46205343414EDB
:106C91005321004E4F204445564943455320464F0A
:106CA100554E44005741524E494E470041444452CB
:106CB10045535320434F554C44004E4F54204245B9
:106CC1002041535349474E45442100257300534504
:106CD1005420444F574E54494C542020203A2025EB
:106CE1002B23352E3166005245414420444F574EE7
:0E6CF10054494C543A20252B23352E31660091
:083325009000F8EEF0A3EFF0B8
:10332D00E4900120F0A3F09005CFF090010DF09006
:10333D00013B74FFF0A3746CF0A37421F07B017A50
:10334D00057969123EF690013B74FFF0A3746CF0A1
:10335D00A37437F07B017A057982123EF690013B1A
:10336D0074FFF0A3746CF0A37437F07B017A0579C8
:10337D009B123EF690013B74FFF0A3746CF0A374A6
:10338D0037F07B017A0579B4123EF6900B1FE0649D
:10339D00016003023765900B5004F0E4900116F0C4
:1033AD00A3F0900116E0FEA3E0FFD39412EE94007B
:1033BD00501C747E2FF582740B3EF583E4F0900162
:1033CD0017E004F070DC900116E004F080D4900B4F
:1033DD0034740BF0A3747EF09001107401F0A3749B
:1033ED0003F0A37404F0E4900118F0A3F09000F939
:1033FD00E024FFFF9000F8E034FFFED3900119E0C8
:10340D009F900118E09E4003023821E4900116F0D0
:10341D00A3F0900116E0FEA3E0FFFD24FAF582E48F
:10342D003400F583E4F0900118E0FAA3E0FBC374D7
:10343D00129BFBE49AFAC3EF9BEE9A400D74FA2DA2
:10344D00F582E43400F58374FFF0900117E004F089
:10345D007006900116E004F0900116E07004A3E0F0
:10346D00641370AEE4900B52F0900116F0A3F0903F
:10347D000B50E0FD900116E0FEA3E0FFC39DEE941E
:10348D000040030237107C007D131226D9900B35B6
:10349D00E02FFF900B34E03E90010EF0A3EFF0E42F
:1034AD0090011AF0A3F090011AE0FEA3E0FFD3946F
:1034BD0009EE940040030236FFEF2430FF90010F18
:1034CD00E02412FD90010EE03400FC900118E0FAAA
:1034DD00A3E0FBC3ED9BFDEC9A8D82F583EFF0909D
:1034ED00013B74FFF0A3746CF0A37438F07B017A88
:1034FD000579B4123EF690011CE4F0A3740BF09024
:10350D00011CE0FEA3E0FF90010EE0FCA3E02FF50F
:10351D0082EC3EF583E0FD74B42FF582E43405F5BD
:10352D0083EDF074B42FF582E43405F583E0700D6E
:10353D0074B42FF582E43405F583745FF090011DAA
:10354D00E004F0700690011CE004F090011CE070A6
:10355D0004A3E0641370A8E49005C7F0127D28124F
:10356D007D5C12000790010EE0FEA3E0AA06F97B38
:10357D0001C003900125EBF0A37400F0A374FAF0E1
:10358D00D003124757900567EEF0A3EFF064014E9C
:10359D00600F900567E07004A3E0640260030236DB
:1035AD00EE9000F9E024FFFF9000F8E034FFFE906C
:1035BD000118E06E7003A3E06F707A900567E070FC
:1035CD0004A3E06401706E90011CF0A3F090011C47
:1035DD00E0FEA3E0FFD39412EE9400504574582FF3
:1035ED00F582E4340BF583E0FD900B52E075F0139A
:1035FD00A4FF900110E0FBA3E0FAA3E02FF9EA3558
:10360D00F0FA90011CE0FEA3E029F9EA3EFAED1272
:10361D0026C790011DE004F070B390011CE004F08A
:10362D0080AB9005CFE004F07B017A0B7958E0FD7B
:10363D007C00125E5E9000F9E024FFFF9000F8E040
:10364D0034FFFEC3900119E09F900118E09E506079
:10365D00E490011CF0A3F090011CE0FEA3E0FFD369
:10366D009412EE9400504990010EE0FCA3E02FF56A
:10367D0082EC3EF583E0FD900B52E075F013A4FF54
:10368D00900110E0FBA3E0FAA3E02FF9EA35F0FA80
:10369D0090011CE0FEA3E029F9EA3EFAED1226C7DF
:1036AD0090011DE004F070AF90011CE004F080A7C4
:1036BD009000F9E024FFFF9000F8E034FFFE900148
:1036CD0018E0B50616A3E0B50711900567E0700484
:1036DD00A3E06402700590010D04F0900B52E0041C
:1036ED00F090011BE004F0700690011AE004F00266
:1036FD0034B3900117E004F07006900116E004F069
:10370D0002347C900B52E0900B50F0900B34E0FEA5
:10371D00A3E0AA06F99001137401F0A3EAF0A3E95E
:10372D00F0900110A3E0FAA3E0FF900B34EAF0A3B0
:10373D00EFF0900113E0F9A3E0FAA3E0900110C9B6
:10374D00F0A3EAF0A3E9F0900119E004F0700690FF
:10375D000118E004F00233FA900118E4F0A3740AA2
:10376D00F09000F8E0FEA3E0FF64024E70089001B7
:10377D0018F0A37464F0D3EF9402EE940040099016
:10378D000118E4F0A374FEF0900116E4F0A304F028
:10379D00900118E0FEA3E0FFD3900117E09F900188
:1037AD0016E09E506F127D5C12000790013B74FF76
:1037BD00F0A3746CF0A37444F0900116E0FFA3E045
:1037CD0090013ECFF0A3EFF07B017A0579B4123E64
:1037DD00F6127D28900116A3E0FF12790990056776
:1037ED00EEF0A3EFF064014E7019900116A3E0FF07
:1037FD009005CFE0FE04F0749E2EF582E43409F5B9
:10380D0083EFF0900117E004F07085900116E0044D
:10381D00F002379D9005CFE0FFD39400400D900549
:10382D0067E4F0A304F0900B50EFF090010DE0B4BD
:10383D000107E4900567F0A3F0900567E07004A31D
:10384D00E06401700302391BE49005CDF0A3F0FF95
:10385D00FE127BC890010DE0640190013B703A743B
:10386D00FFF0A3746CF0A37452F07B017A057969B3
:10387D00123EF690013B74FFF0A3746CF0A37469D3
:10388D00F07B017A057982123EF690013B74FFF0D0
:10389D00A3746CF0A3747F803874FFF0A3746CF084
:1038AD00A37494F07B017A057969123EF690013B81
:1038BD0074FFF0A3746CF0A37437F07B017A057973
:1038CD0082123EF690013B74FFF0A3746CF0A3746A
:1038DD0037F07B017A05799B123EF6E4900B50F0A0
:1038ED00900B52F09005CFF090013B74FFF0A37454
:1038FD006CF0A37437F07B017A0579B4123EF612A1
:10390D007D281200077FE87E0312786D80129005E6
:10391D00CF7401F0FF12684190011EE4F0A3EFF0A7
:08392D00900567E0FEA3E0FF36
:01393500226F
:0B475700900122EBF0A3EAF0A3E9F0D0
:10476200E4900567F0A3F0901543F0A374BFF090B6
:1047720011AFE4F0A374FFF090154CE0FEA3E0FF4C
:10478200F5828E837481F08F828E83A374F0F08F12
:10479200828E83A3A3742AF08F828E83A3A3A37431
:1047A20001F0EF2404F582E43EF5837413F0E49003
:1047B2000128F0A3F0900122E0FBA3E0FAA3E0F9C4
:1047C200900128E0FEA3E0FFF5828E8312269AFD77
:1047D200EF2405FFE43EFE90154CE0FAA3E02FF52E
:1047E20082EA3EF583EDF0900129E004F070069034
:1047F2000128E004F0900128E07004A3E064137043
:10480200B490154CE0FEA3E0FF2418F582E43EF5D7
:10481200837403F0EF2419F582E43EF5837413F0F8
:10482200E4900128F0A3F0900125E0FBA3E0FAA3B5
:10483200E0F9A3E0FEA3E0FFF5828E8312269AFD43
:10484200EF241AFFE43EFE90154CE0FAA3E02FF5A8
:1048520082EA3EF583EDF0900129E004F0700690C3
:104862000128E004F0900128E07004A3E0641370D2
:10487200B6901413E4F0A3742DF0124E361253BD09
:10488200EF4E7007900567F0A304F090097CE0708A
:1048920004A3E064017040901541E07004A3E06459
:1048A20073707A90154CE0FCA3E0F5828C83E0FDF6
:1048B20090154AE0FAA3E0FBF5828A83E0B505157C
:1048C20090154CA3E0F5828C83A3E0FD8B828A8352
:1048D200A3E06D604F8046901543E0FCA3E0FD909D
:1048E2001541E06C7003A3E06D703290154CE0FC52
:1048F200A3E0F5828C83E0FD90154AE0FAA3E0FB89
:10490200F5828A83E0B5051590154CA3E0F5828CFB
:1049120083A3E0FD8B828A83A3E06D6007E49005A8
:1049220067F0A3F0EF30E209900567E4F0A37402A8
:10493200F0900567E0FEA3E0FF4E70012290154A59
:10494200E0FEA3E0F5828E83A3A3E0FF90012CE4B6
:10495200F0A3EFF07F037E0090012DE02402FD9092
:10496200012CE03400FCC3EF9DEE9C4003024B524D
:1049720090154AE0FCA3E0F5828C830FEFAC067041
:10498200010E14FDE5822DF582E5833CF583E0FD01
:104992007C0090154AE0FAA3E0F5828A830FEFAA21
:1049A2000670010E14FBE5822BF582E5833AF5834E
:1049B200E0FB90012AE4F0A3EBF0EC709BED24FE07
:1049C200607824FE7003024A7124FE7003024ABC1E
:1049D20024FD7003024B182408600302495AE49034
:1049E2000128F0A3F090012AE0FCA3E0FD90012849
:1049F200E0FAA3E0FBC39DEA9C400302495A9015EA
:104A02004AE0FCA3E0F5828C830FEFAC0670010E46
:104A120014FDE5822DF582E5833CF583E0FD7458B3
:104A22002BF582E4340BF583EDF0900129E004F0DC
:104A320070B3900128E004F080AB90097CE0700430
:104A4200A3E06401600302495A90154AE0FCA3E026
:104A5200F5828C830FEFAC0670010E14FDE5822DFA
:104A6200F582E5833CF583E0FD90012E024B4A90EE
:104A7200154AE0FCA3E0F5828C830FEFAC067001CF
:104A82000E14FDE5822DF582E5833CF583E0FD9071
:104A92000B72E4F0A3EDF0900B72E0FCA3E0FD6476
:104AA200014C700302495AED64114C700302495AD9
:104AB200E4900567F0A3F002495AE4900128F0A3BC
:104AC200F090012AE0FCA3E0FD900128E0FAA3E0C7
:104AD200FBC39DEA9C400302495A90154AE0FCA39D
:104AE200E0F5828C830FEFAC0670010E14FDE582B7
:104AF2002DF582E5833CF583E0FD74652BF582E4B8
:104B02003405F583EDF0900129E004F070B39001D3
:104B120028E004F080AB90097CE07004A3E064011B
:104B2200600302495A90154AE0FCA3E0F5828C83A7
:104B32000FEFAC0670010E14FDE5822DF582E583C0
:104B42003CF583E0FD900130E4F0A3EDF002495A18
:084B5200900567E0FEA3E0FFFF
:014B5A002238
:105E5E00900122EBF0A3EAF0A3E9F0A3ECF0A3ED9E
:015E6E00F043
:105E6F00901543E4F0A37453F09011AFECF0A3ED51
:105E7F00F0E4901413F0A3F0124E361253BD9001BC
:105E8F0028EFF0901543E4F0A374BFF09011AFE446
:105E9F00F0A374FFF07F1390154CE0FCA3E0FDF529
:105EAF00828C837481F08D828C83A374F0F08D8249
:105EBF008C83A3A37418F08D828C83A3A3A3740186
:105ECF00F090154CE0FCA3E02404F582E43CF5834C
:105EDF00EFF0E4900127F0900122E0FBA3E0FAA39A
:105EEF00E0F9900127E0FFF58275830012269AFEF4
:105EFF00EF2405FDE433FC90154CE0FAA3E02DF5FB
:105F0F0082EA3CF583EEF0900127E004F0E0B41351
:105F1F00C690154CE0FEA3E0FF2418F582E43EF591
:105F2F00837402F0EF2419F582E43EF5837401F0D7
:105F3F00900125A3E0FF90154CE0FCA3E0241AF597
:105F4F0082E43CF583EFF0901413E4F0A3741BF09C
:105F5F00124E361253BD900128EFF07003026019F4
:105F6F00E4900567F0A3F0900127F0900127E0FF80
:105F7F00D39412503EE0FE2458F582E4340BF5839F
:105F8F00E0FD74692EF582E43405F583EDF0746954
:105F9F002FF582E43405F583E07010900127E0249B
:105FAF0069F582E43405F583745FF0900127E0040E
:105FBF00F080B8E490057CF090013B74FFF0A3747F
:105FCF006CF0A374A5F07B017A057982123EF690EE
:105FDF00013B74FFF0A3746CF0A374ADF07B017AF6
:105FEF0005799B123EF690013B74FFF0A3746CF0A1
:105FFF00A374BBF07B017A0579B4123EF6127D28AB
:0A600F001200077FDC7E0512786D99
:016019002264
:084B5B00900124EEF0A3EFF03D
:104B63009011AFEEF0A3EFF0901543E4F0A37412AD
:104B7300F09011B3E4F0A374EAF0E4901413F0A3FB
:104B8300F0125650900124E0FFA3E09011AFCFF054
:104B9300A3EFF0901543E4F0A37412F09011B3E483
:104BA300F0A37405F0E4901413F0A3F0125650EF41
:104BB3004E6003024E35900126E4F0A304F09015F5
:104BC3004AE0FEA3E0F5828E83C083C08290012673
:104BD300E475F001122776FED082D083E58225F0BA
:104BE300F582E5833EF583E0FF7E00E4FDFCC3ED43
:104BF3009FEC9E505A90154AE0FAA3E0F5828A830F
:104C0300C083C082900126E475F001122776FAD0A2
:104C130082D083E58225F0F582E5833AF583E0FBD4
:104C2300AA05748A2AF582E43409F583EBF0748AC1
:104C33002AF582E43409F583E0700D748A2AF5823B
:104C4300E43409F5837420F00DBD00010C809F74DA
:104C53008A2FF582E43409F583E4F090154AE0FEE7
:104C6300A3E0F5828E83C083C082900126E475F0B1
:104C730001122776FED082D083E58225F0F582E506
:104C8300833EF583E0FF7E00E4FCFDC3ED9FEC9ED5
:104C9300505A90154AE0FAA3E0F5828A83C083C094
:104CA30082900126E475F001122776FAD082D08330
:104CB300E58225F0F582E5833AF583E0FBAA0574E6
:104CC300C02AF582E43409F583EBF074C02AF58237
:104CD300E43409F583E0700D74C02AF582E43409E5
:104CE300F5837420F00DBD00010C809F74C02FF577
:104CF30082E43409F583E4F090154AE0FEA3E0F57D
:104D0300828E83C083C082900126E475F00112274E
:104D130076FED082D083E58225F0F582E5833EF5E9
:104D230083E0FF7E00E4FCFDC3ED9FEC9E505A90B0
:104D3300154AE0FAA3E0F5828A83C083C08290011A
:104D430026E475F001122776FAD082D083E5822516
:104D5300F0F582E5833AF583E0FBAA0574202AF592
:104D630082E4340BF583EBF074202AF582E4340BF0
:104D7300F583E0700D74202AF582E4340BF5837417
:104D830020F00DBD00010C809F74202FF582E434C8
:104D93000BF583E4F090154AE0FEA3E0F5828E83E1
:104DA300C083C082900126E475F001122776FED0FD
:104DB30082D083E58225F0F582E5833EF583E0FF2B
:104DC3007E00E4FCFDC3ED9FEC9E505A90154AE033
:104DD300FAA3E0F5828A83C083C082900126E4753A
:104DE300F001122776FAD082D083E58225F0F5828E
:104DF300E5833AF583E0FBAA05743C2AF582E434A3
:104E03000BF583EBF0743C2AF582E4340BF583E075
:104E1300700D743C2AF582E4340BF5837420F00D95
:104E2300BD00010C809F743C2FF582E4340BF583A5
:024E3300E4F0A9
:014E3500225A
:1058DF00E49000F9F0A3F01218A69000F9EEF0A3EF
:1058EF00EFF04E6003025AD2126715E49000F8F001
:1058FF009000F8E0FFFDD3900B77E09D900B76E0E2
:10590F009400406BEF75F00CA424D8F9740735F0B0
:10591F00FA7B01C0019000F8E075F019A424DAF9C0
:10592F00740935F0A801FC7D01D001122A6E900098
:10593F00F8E075F019A424DAF9740935F0FA7B014F
:10594F00C003C002C001E075F014A42474F97408F8
:10595F0035F0FA9000FEEBF0A3EAF0A3E9F0D001E6
:10596F00D002D0031276239000F8E004F0808190EB
:10597F000B7CE4F0A304F0E49000F8F09000F8E062
:10598F00FFC39413503EE0FE2458F582E4340BF528
:10599F0083E0FD74692EF582E43405F583EDF07430
:1059AF00692FF582E43405F583E070109000F8E07C
:1059BF002469F582E43405F583745FF09000F8E014
:1059CF0004F080B8E490057CF090013B74FFF0A3E5
:1059DF00746CF0A374CCF0A37401F0A37409F0A35A
:1059EF0074DAF07B017A057982123EF69005CFE0EA
:1059FF00FF1269509000F9EEF0A3EFF04E60030232
:105A0F005AD2900982E0FCA3E0FDA3E0FEA3E0FFE1
:105A1F00900986122913E4FFFE7DC87C4290098607
:105A2F00E0F8A3E0F9A3E0FAA3E0FB1221071223A9
:105A3F0058AB07AA067C007D19122740C3EB9DFDCA
:105A4F00EA9CFC12231F900986122913900986E005
:105A5F00FCA3E0FDA3E0FEA3E0FFE4FBFA79C87826
:105A6F004212221090098612291390013B74FFF005
:105A7F00A3746CF0A374CFF0900986E0FCA3E0FD53
:105A8F00A3E0FEA3E0FF90013E1229137B017A05EC
:105A9F00799B123EF690013B74FFF0A3746CF0A358
:105AAF0074E8F0900982E0FCA3E0FDA3E0FEA3E020
:105ABF00FF90013E1229137B017A0579B4123EF64D
:0B5ACF00127D289000F9E0FEA3E0FF2C
:015ADA0022A9
:05684100900122EFF0C0
:10684600900B1FE06401704EFF900B34E0FCA3E058
:10685600F5828C83C083C082900122E024FFFDE490
:1068660034FFFCD082D08375F013ED122950EC75FD
:10687600F013A42583F583E5822FF582E43583F5AD
:1068860083E0FE74582FF582E4340BF583EEF00FA7
:10689600EFB413B58012900122E0249DF582E43412
:1068A60009F583E0FF126B40901543E4F0A37412E0
:1068B600F0900122E0FF9011AFE4F0A3EFF0900911
:1068C6007CE07004A3E06401701C9011B3F0A37423
:1068D60008F0E4901413F0A3F0125650900123EF41
:1068E600F06003E0FF22900122E0FF7E00124B5B86
:1068F600900B74E4F0A304F090097CE07004A3E02C
:10690600640270329011B3F0A37488F0E49014130B
:10691600F0A3F0125650900123EFF06003E0FF223F
:1069260090154AE0FEA3E0F5828E83A3E0FF900B6C
:1069360074E4F0A3EFF0900B3AE4F0A304F0FF7ECA
:0969460000127BC8900123E0FF60
:01694F002225
:10790900E4900567F0A3F0901543F0A37493F09009
:1079190011AFE4F0A3EFF0E4901413F0A3F0124ECA
:10792900361253BDEF4E7007900567F0A304F0902F
:107939001541E07004A3E064736007E4900567F003
:0A794900A3F0900567E0FEA3E0FF45
:017953002211
:106B4000901543E4F0A374BFF09011AFE4F0A3EF0D
:106B5000F090154CE0FEA3E0FFF5828E837481F087
:106B60008F828E83A374F0F08F828E83A3A3742A06
:106B7000F08F828E83A3A3A37401F0EF2404F58227
:106B8000E43EF5837413F0E4FFEF2405FDE433FCE9
:106B900090154CE0FAA3E02DF582EA3CF583E4F091
:106BA0000FEFB413E490154CE0FEA3E0FF2418F5BA
:106BB00082E43EF5837403F0EF2419F582E43EF598
:106BC000837413F0E4FFEF241AFDE433FC90154CBA
:106BD000E0FAA3E02DF582EA3CF583E4F00FEFB490
:106BE00013E4901413E4F0A3742DF0124E361253F4
:106BF000BD900124EFF0E4FFEF2405FDE433FC90A9
:106C0000154AE0FAA3E02DF582EA3CF583E0FE7434
:106C1000582FF582E4340BF583EEF00FEFB413D860
:016C20002251
:10648F00E47B0CFAF9F8900B6EE0FCA3E0FDA3E0BF
:10649F00FEA3E0FF12284F90019812291390019844
:1064AF00E0FCA3E0FDA3E0FEA3E0FFE412231AA8A3
:1064BF0004A905AA06AB07E4FFFE7D807C3F1222EC
:1064CF0010900101122913900101E0F8A3E0F9A344
:1064DF00E0FAA3E0FB7F6F7E127D837C3A122210DD
:1064EF00122358900198122913900198E0F8A3E015
:1064FF00F9A3E0FAA3E0FBC3E49BFFE49AFE740167
:10650F0099FDE498FC900198122913900101E0F88D
:10651F00A3E0F9A3E0FAA3E0FB7F0A7ED77D237CFB
:10652F003C12221012235890019C12291390019CA7
:10653F00E0F8A3E0F9A3E0FAA3E0FBC3E49BFFE4D8
:10654F009AFE740199FDE498FC90019C1229139016
:10655F00019CE0FCA3E0FDA3E0FEA3E0FFE4122317
:10656F001A900101E0F8A3E0F9A3E0FAA3E0FB120F
:10657F002107A804A905AA06AB077F0A7ED77DA32A
:10658F007C3C1222109000FD1229139000FDE0FCBC
:10659F00A3E0FDA3E0FEA3E0FF122358900196EEC7
:1065AF00F0A3EFF0FDAC06E412231F9000FDE0F81E
:1065BF00A3E0F9A3E0FAA3E0FB1222AD6010400EB6
:0E65CF00900197E004F07006900196E004F051
:0165DD00229B
:107C2E00AF89EF60047E0180027E00AF067F018F78
:107C3E0089900198A3A3A3E0F58A900198E0FCA394
:0F7C4E00E0FDA3E0FEA3E0FF78081229008F8C71
:017C5D002204
:03000B0002781068
:10781000C0E0C0F0C083C082C0D075D000C000C03E
:1078200001C002C003C004C005C006C007C28C90DE
:107830000198A3A3A3E0F58A900198E0FCA3E0FDE2
:10784000A3E0FEA3E0FF78081229008F8C127CDCF5
:10785000D28CD007D006D005D004D003D002D001FE
:0D786000D000D0D0D082D083D0F0D0E03264
:107B9300AF89C28EEF540F4410F58990019CA3A3C3
:107BA300A3E0F58B90019CE0FCA3E0FDA3E0FEA322
:107BB300E0FF78081229008F8DD209E4900B6CF056
:047BC300A3F0D28ECB
:017BC700229B
:08786D00900135EEF0A3EFF0ED
:10787500E4A3F0A3F08037900135E0FEA3E0FF7CA0
:10788500007D0C1226EB7C007D0A1226D9D39001CF
:1078950038E09F900137E09E501A120007200AD762
:1078A500900138E004F07006900137E004F0D20A48
:0678B500D28C80C3C28CDE
:0178BB0022AA
:107CDC00D3900B57E09401900B56E09400500DA3F9
:107CEC00E004F07010900B56E004F022C20AE4900D
:067CFC000B56F0A3F0227C
:107C5E00900196E0FEA3E0FFD3900B6DE09F900B9A
:107C6E006CE09E500FA3E004F07006900B6CE004E5
:107C7E00F0D28E22C209E4900B6CF0A3F0C28E22D9
:03001B0002795413
:10795400C0E0C083C082C0D075D000C000C004C0E5
:1079640005C006C007C28E90019CA3A3A3E0F58BBB
:1079740090019CE0FCA3E0FDA3E0FEA3E0FF7808F7
:107984001229008F8D127C5ED007D006D005D0045A
:0B799400D000D0D0D082D083D0E032F1
:107210000000000F00200022002A002E0030003263
:10722000000000000000000000000000000000005E
:1072300000320041005200530057005B005C005DCB
:10724000005E0000000000000000000000000000E0
:10725000005E00640069008900A900AB00AD000079
:107260000000000F0020002200250028002A002C2A
:10727000000000000000000000000000000000000E
:10728000002C0031004C004D0051005500560057B5
:107290000058000000000000000000000000000096
:1072A0000058005E0063006F0073007500760000F8
:103953004409784320000042097E000142098000A7
:10396300074209D600114209D800184209BE0021B6
:0C3973004209D40026420B76000DC10B67
:107455004D444C3A2000532F4E3A200042414E44B1
:10746500533A20004245414D57494454483A20007B
:107475004741494E3A20004D415854494C543A2011
:10748500004D494E54494C543A2000444154453A24
:107495002000494E5354414C2049443A200042545F
:1074A500532049443A2000534543544F523A200053
:1074B50042454152494E473A20004D4543485449BB
:0574C5004C543A2000C8
:1067150090013B74FFF0A37474F0A37455F07B01F2
:106725007A0779D8123EF690013B74FFF0A3747492
:10673500F0A3745BF07B017A0779E4123EF69001D1
:106745003B74FFF0A37474F0A37461F07B017A07C6
:1067550079F0123EF690013B74FFF0A37474F0A338
:106765007469F07B017A0779FC123EF690013B745F
:10677500FFF0A37474F0A37475F07B017A087908AF
:10678500123EF690013B74FFF0A37474F0A3747C81
:10679500F07B017A087914123EF690013B74FFF004
:1067A500A37474F0A37486F07B017A087920123EF5
:1067B500F690013B74FFF0A37474F0A37490F07B22
:1067C500017A08792C123EF690013B74FFF0A37410
:1067D50074F0A37497F07B017A087938123EF6902D
:1067E500013B74FFF0A37474F0A374A3F07B017AEA
:1067F500087944123EF690013B74FFF0A37474F0DF
:10680500A374ACF07B017A087950123EF690013BF7
:1068150074FFF0A37474F0A374B5F07B017A087962
:106825005C123EF690013B74FFF0A37474F0A37400
:0C683500BFF07B017A087968123EF62261
:10768E00257300414E54454E4E41204E4F540052EC
:10769E004553504F4E44494E472E2050524553535A
:1076AE002046494E4400464F52204E4558542041E4
:1076BE004E54454E4E4100414E54454E4E41204E85
:1076CE004F5420524541445900005741524E494EA5
:1076DE0047004144445245535320434F4E464C4974
:0376EE0043540002
:106F6A00E49000F8F0FF74B42FF582E43405F58359
:106F7A00E0FE74F92FF582E43400F583EEF00FEFAA
:106F8A00B419E3901542E030E00302701490154AF8
:106F9A00E0FCA3E0F5828C83E0640B706D9000F84E
:106FAA0004F090013B74FFF0A37476F0A3748EF0A2
:106FBA0090154AE0FEA3E0F5828E83A3E075F019EE
:106FCA00A424DEF9740D35F0FA90013E7401F0A3A1
:106FDA00EAF0A3E9F07B017A0579B4123EF6127D54
:106FEA00287FF47E0112786DE4FF74F92FF582E4AC
:106FFA003400F583E0FE74B42FF582E43405F5839A
:0F700A00EEF00FEFB419E3127D289000F8E0FFCD
:017019002254
:10565000900128E4F0A304F090012CE4F0A304F0FE
:10566000120007E490012AF0A3F0901544E030E026
:1056700003025701901543E4F0A37493F09005CF13
:10568000E0FFFD9011AFE4F0A3EDF0900B1FE07090
:1056900014749D2FF582E43409F583E0FF9011AF77
:1056A000E4F0A3EFF0901413E0FFA3E0900130CFFB
:1056B000F0A3EFF0E4901413F0A3F0124E3612535F
:1056C000BD90012EEEF0A3EFF0A3E0FFA3E0901455
:1056D00013CFF0A3EFF0901543E4F0A37412F09011
:1056E0000B58E064416009901543E4F0A37410F096
:1056F000900B59E064526009901543E4F0A37410D4
:10570000F0900B1FE070179005CFE0249DF582E428
:105710003409F583E0FF9011AFE4F0A3EFF0124EEF
:10572000361253BD90012EEEF0A3EFF04E602090A4
:10573000012DE004F0700690012CE004F0D39001FC
:105740002DE0940390012CE094005003025660E495
:10575000FF74582FF582E4340BF583E0FE74692F53
:10576000F582E43405F583EEF074692FF582E434B4
:1057700005F583E0700D74692FF582E43405F58337
:10578000745FF00FEFB413C9E490057CF090012E24
:10579000E07002A3E0605390012AE4F0A304F090CB
:1057A000013B74FFF0A37476F0A37491F07B017A4F
:1057B000057982123EF690013B74FFF0A37476F0F7
:1057C000A3749DF07B017A05799B123EF690013B14
:1057D00074FFF0A37476F0A374B4F07B017A0579BA
:1057E000B4123EF6127D280258D6901541E070049E
:1057F000A3E064357055900B51E0704F90012AF092
:10580000A304F090013B74FFF0A37476F0A374C579
:10581000F07B017A057982123EF690013B74FFF02D
:10582000A37476F0A374D7F07B017A05799B123EBE
:10583000F690013B74FFF0A37476F0A374D7F07B6D
:10584000017A0579B4123EF6127D289011AFE0FE80
:10585000A3E0FF9011ADE06E7003A3E06F6059907C
:10586000012EE07002A3E0704F90012AF0A304F033
:1058700090013B74FFF0A37476F0A374D8F07B0121
:105880007A057982123EF690013B74FFF0A374769C
:10589000F0A374E0F07B017A05799B123EF690014B
:1058A0003B74FFF0A37476F0A374D7F07B017A0504
:1058B00079B4123EF6127D28901542E020E0179050
:1058C000154AE0FEA3E0F5828E83E0B40B08900158
:0E58D0002AE4F0A304F090012AE0FEA3E0FF1A
:0158DE0022A7
:107AEB0025750025752C25752C25750025752C25E0
:107AFB00752C25752C2575002523342E3266002513
:107B0B002B23342E326600256325632F25632563D3
:097B1B002F25632563002573008A
:1018A6009005CFE0FF9011AFE4F0A3EFF0900B743A
:1018B600E07004A3E064016003021A42901413F07E
:1018C600A3F090097EE0F508A3E0F509C39009812D
:1018D600E09509900980E09508403690154CE0FCAB
:1018E600A3E0F5828C83C083C082901413E475F064
:1018F60001122776FCD082D083E58225F0F582E5B9
:10190600833CF583E509F00509E50970BF05088004
:10191600BB901543E4F0A37412F09011B3E4F0A366
:10192600740FF01256508E0E8F0FE50F450E6001A4
:1019360022E4F510F51190154AE0FCA3E02511F517
:1019460082EC3510F583E0751200F5130511E511EB
:1019560070020510FF90154AE0FCA3E02FF582EC1B
:101966003510F583E0751400F51524FFFFE51434F2
:10197600FFFEEF25E0FFEE33FE900B53E0FBA3E006
:10198600FAA3E0F98F828E8312278CFDACF0E51561
:1019960025E0FFE514338F82F58312278CAEF0C362
:1019A6009DF50BEE9CF50A750800750901D3E5094E
:1019B600950BE508950A5067E51524FFFFE51434F5
:1019C600FFFEEF25E0FFEE33FE900B53E0FBA3E0B6
:1019D600FAA3E0F98F828E8312278CFF2509CFE5C3
:1019E6000835F0CF24FFF50DEF34FFF50C0511E5B2
:1019F6001170020510FF90154AE0FCA3E02FF58256
:101A0600EC3510F583E0FF74D0250DF582740535AD
:101A16000CF583EFF00509E50970920508808E90B4
:101A26001412E024FFFF901411E034FFFEC3E51109
:101A36009FE5109E5003021952021BF2E490141304
:101A4600F0A3F0900B3AA3E0FF90154CE0FCA3E066
:101A5600F5828C83C083C082901413E475F0011262
:101A66002776FCD082D083E58225F0F582E5833C9B
:101A7600F583EFF090097EE0F508A3E0F509C39041
:101A86000981E09509900980E09508403690154C4B
:101A9600E0FCA3E0F5828C83C083C082901413E43B
:101AA60075F001122776FCD082D083E58225F0F509
:101AB60082E5833CF583E509F00509E50970BF0574
:101AC6000880BB901543E4F0A37412F09011B3E4C0
:101AD600F0A37484F01256508E0E8F0FE50F450E4C
:101AE60060012275100075110190154AE0FCA3E013
:101AF6002511F582EC3510F583E0751200F5130516
:101B060011E51170020510FF90154AE0FCA3E02FC5
:101B1600F582EC3510F583E0751400F51524FFFF0A
:101B2600E51434FFFEEF25E0FFEE33FE900B53E0A5
:101B3600FBA3E0FAA3E0F98F828E8312278CFDAC1B
:101B4600F0E51525E0FFE514338F82F58312278C27
:101B5600AEF0C39DF50BEE9CF50A750800750901FC
:101B6600D3E509950BE508950A5067E51524FFFFAF
:101B7600E51434FFFEEF25E0FFEE33FE900B53E055
:101B8600FBA3E0FAA3E0F98F828E8312278CFF2550
:101B960009CFE50835F0CF24FFF50DEF34FFF50C3E
:101BA6000511E51170020510FF90154AE0FCA3E04F
:101BB6002FF582EC3510F583E0FF74D0250DF58204
:101BC6007405350CF583EFF00509E50970920508F3
:101BD600808E901412E024FFFF901411E034FFFE73
:101BE600C3E5119FE5109E5003021B05900B74E0A0
:101BF6007004A3E064016003021D81901413F0A336
:101C0600F09009BEE0F508A3E0F509C39009D5E018
:101C160095099009D4E09508403690154CE0FCA350
:101C2600E0F5828C83C083C082901413E475F001C2
:101C3600122776FCD082D083E58225F0F582E583F3
:101C46003CF583E509F00509E50970BF050880BB89
:101C5600901543E4F0A37412F09011B3E4F0A3746A
:101C66000FF01256508E0E8F0FE50F450E600122B3
:101C7600E4F510F51190154AE0FCA3E02511F58274
:101C8600EC3510F583E0751200F5130511E51170BA
:101C9600020510FF90154AE0FCA3E02FF582EC3513
:101CA60010F583E0751400F51524FFFFE51434FFE5
:101CB600FEEF25E0FFEE33FE900B53E0FBA3E0FAC8
:101CC600A3E0F98F828E8312278CFDACF0E51525F3
:101CD600E0FFE514338F82F58312278CAEF0C39DA7
:101CE600F50BEE9CF50A750800750901D3E5099513
:101CF6000BE508950A5067E51524FFFFE51434FF48
:101D0600FEEF25E0FFEE33FE900B53E0FBA3E0FA77
:101D1600A3E0F98F828E8312278CFF2509CFE50871
:101D260035F0CF24FFF50DEF34FFF50C0511E51165
:101D360070020510FF90154AE0FCA3E02FF582EC37
:101D46003510F583E0FF74D0250DF5827405350C4A
:101D5600F583EFF00509E50970920508808E901469
:101D660012E024FFFF901411E034FFFEC3E5119F3B
:101D7600E5109E5003021C91021F31E4901413F0EB
:101D8600A3F0900B3AA3E0FF90154CE0FCA3E0F51E
:101D9600828C83C083C082901413E475F0011227ED
:101DA60076FCD082D083E58225F0F582E5833CF58A
:101DB60083EFF09009BEE0F508A3E0F509C39009AA
:101DC600D5E095099009D4E09508403690154CE089
:101DD600FCA3E0F5828C83C083C082901413E47563
:101DE600F001122776FCD082D083E58225F0F582B9
:101DF600E5833CF583E509F00509E50970BF0508AB
:101E060080BB901543E4F0A37412F09011B3E4F094
:101E1600A37484F01256508E0E8F0FE50F450E6098
:101E2600012275100075110190154AE0FCA3E0250A
:101E360011F582EC3510F583E0751200F5130511E6
:101E4600E51170020510FF90154AE0FCA3E02FF59E
:101E560082EC3510F583E0751400F51524FFFFE5D7
:101E66001434FFFEEF25E0FFEE33FE900B53E0FB4C
:101E7600A3E0FAA3E0F98F828E8312278CFDACF0E3
:101E8600E51525E0FFE514338F82F58312278CAE26
:101E9600F0C39DF50BEE9CF50A750800750901D394
:101EA600E509950BE508950A5067E51524FFFFE55A
:101EB6001434FFFEEF25E0FFEE33FE900B53E0FBFC
:101EC600A3E0FAA3E0F98F828E8312278CFF2509FF
:101ED600CFE50835F0CF24FFF50DEF34FFF50C05FF
:101EE60011E51170020510FF90154AE0FCA3E02FE2
:101EF600F582EC3510F583E0FF74D0250DF582747C
:101F060005350CF583EFF00509E5097092050880A3
:101F16008E901412E024FFFF901411E034FFFEC3EC
:101F2600E5119FE5109E5003021E447F017E0012BC
:051F36000036E4FEFF8F
:011F3B002283
:080036009000FBEEF0A3EFF0D7
:10003E0064014E6003020E43900101F0A3F0E0252F
:10004E00E0FF900101E033FE900B53E0FBA3E0FADA
:10005E00A3E0F98F828E8312278CFF900103E5F0C7
:10006E00F0A3EFF0E42401FFE433FEEF25E0FFEE12
:10007E00338F82F58312278CFDACF0900102E025C0
:10008E00E0FF900101E0338F82F58312278CFFC3CE
:10009E00ED9FFEEC95F0900105F0A3CEF0E4A3F0F9
:1000AE00A3F0900105E0FEA3E0FFA3E0FCA3E0FDBA
:1000BE00C39FEC9E400302016C900103E0FEA3E09F
:1000CE0024D0F58274053EF583E0FF900101E0FA3D
:1000DE00A3E0FB90087475F014122950EA75F01421
:1000EE00A42583F583E5822DF582E5833CF583EF28
:1000FE00F090087475F014EB122950EA75F014A400
:10010E002583F583E5822DF582E5833CF583E0704A
:10011E002E900107E0FEA3E0FF900101E0FCA3E0BA
:10012E0090087475F014122950EC75F014A4258300
:10013E00F583E5822FF582E5833EF5837420F090FA
:10014E000104E004F07006900103E004F090010851
:10015E00E004F07006900107E004F00200B0900198
:10016E0005E0FEA3E0FF900101E0FCA3E09008741F
:10017E0075F014122950EC75F014A42583F583E55F
:10018E00822FF582E5833EF583E4F0900101F0A322
:10019E0004F0E025E0FF900101E033FE900B53E008
:1001AE00FBA3E0FAA3E0F98F828E8312278CFF90D7
:1001BE000103E5F0F0A3EFF0740125E0FFE433FE58
:1001CE00EF25E0FFEE338F82F58312278CFDACF026
:1001DE00900102E025E0FF900101E0338F82F5836C
:1001EE0012278CFFC3ED9FFEEC95F0900105F0A356
:1001FE00CEF0E4A3F0A3F0900105E0FEA3E0FFA390
:10020E00E0FCA3E0FDC39FEC9E40030202C19001FF
:10021E0003E0FEA3E024D0F58274053EF583E0FFF3
:10022E00900101E0FAA3E0FB90087475F014122916
:10023E0050EA75F014A42583F583E5822DF582E549
:10024E00833CF583EFF090087475F014EB1229508F
:10025E00EA75F014A42583F583E5822DF582E583F6
:10026E003CF583E0702E900107E0FEA3E0FF9001C5
:10027E0001E0FCA3E090087475F014122950EC759F
:10028E00F014A42583F583E5822FF582E5833EF5F0
:10029E00837420F0900104E004F07006900103E0F6
:1002AE0004F0900108E004F07006900107E004F0FD
:1002BE00020205900105E0FEA3E0FF900101E0FCC3
:1002CE00A3E090087475F014122950EC75F014A484
:1002DE002583F583E5822FF582E5833EF583E4F0F1
:1002EE00900101F0A37402F0E025E0FF900101E01F
:1002FE0033FE900B53E0FBA3E0FAA3E0F98F828E5E
:10030E008312278CFF900103E5F0F0A3EFF090012C
:10031E0003E0FCA3E0FD24D1F58274053CF583E0F7
:10032E009000FFF0A3E4F074D02DF58274053CF537
:10033E0083E0FF900100E02FFE9000FFE03400907C
:10034E0000FDF0A3CEF0900101E0FEA3E0FF7C00E3
:10035E007D141226D974742FF974083EFA7B01901D
:10036E00013B74FFF0A3747AF0A374EBF09000FDE0
:10037E00E0FFA3E090013ECFF0A3EFF0123EF69027
:10038E000101E4F0A37403F0E025E0FF900101E029
:10039E0033FE900B53E0FBA3E0FAA3E0F98F828EBD
:1003AE008312278CFF900103E5F0F0A3EFF07403A6
:1003BE002401FFE433FEEF25E0FFEE338F82F58359
:1003CE0012278CFDACF0900102E025E0FF900101B8
:1003DE00E0338F82F58312278CFFC3ED9FFEEC95E1
:1003EE00F0900105F0A3CEF0E4A3F0A3F090097C09
:1003FE00E0FCA3E0FD64014C6018900103E0FEA355
:10040E00E024D1F58274053EF583E09000FFF0A361
:10041E00E4F0900103E0FEA3E024D0F58274053EE3
:10042E00F583E0FF900100E02FFB9000FFE0340029
:10043E00FA900108E025E0FF900107E033FE740B0F
:10044E002FF58274013EF583EAF0A3EBF0900104E0
:10045E00E004F07006900103E004F0ED64014C60DE
:10046E000E900104E004F07006900103E004F09099
:10047E000108E004F07006900107E004F090010717
:10048E00E07004A3E0640460030203FB90097CE0C7
:10049E007004A3E064017057900101E0FEA3E0FF39
:1004AE007C007D141226D974742FF974083EFA7BE1
:1004BE000190013B74FFF0A3747AF0A374EEF090F8
:1004CE00010BE0FFA3E090013ECFF0A3EFF090010F
:1004DE000DE0FFA3E0900140CFF0A3EFF090010FED
:1004EE00E0FFA3E0900142CFF0A3EFF0123EF690B2
:1004FE00097CE07004A3E06402706E900101E0FEDE
:10050E00A3E0FF7C007D141226D974742FF97408B1
:10051E003EFA7B01C003C00290013B74FFF0A3744E
:10052E007AF0A374F7F090010BE0FFA3E090013E88
:10053E00CFF0A3EFF090010DE0FFA3E0900140CFCC
:10054E00F0A3EFF090010FE0FFA3E0900142CFF097
:10055E00A3EFF0900111E0FFA3E0900144CFF0A3D0
:10056E00EFF0D002D003123EF6900101E4F0A37436
:10057E0004F0E025E0FF900101E033FE900B53E024
:10058E00FBA3E0FAA3E0F98F828E8312278CFF90F3
:10059E000103E5F0F0A3EFF0900103E0FEA3E024E9
:1005AE00D0F58274053EF583E0FCE41223247BCD66
:1005BE007ACC79CC783D122107900128122913901C
:1005CE000103E0FEA3E024D1F58274053EF583E03D
:1005DE00FCE41223247BCD7ACC79CC783D12210712
:1005EE0090012C122913900103E0FEA3E024D2F512
:1005FE008274053EF583E0FCE41223247BCD7ACC95
:10060E0079CC783D12210790013012291390097C84
:10061E00E07004A3E064016027900103E0FEA3E014
:10062E0024D3F58274053EF583E0FCE41223247B8B
:10063E00CD7ACC79CC783D12210790013412291352
:10064E00900101E0FEA3E0FF7C007D141226D97418
:10065E00742FF974083EFA7B0190013B74FFF0A3EE
:10066E00747BF0A37403F0900128E0FCA3E0FDA3DB
:10067E00E0FEA3E0FF90013E122913123EF6900118
:10068E0001E4F0A37405F0E025E0FF900101E033F2
:10069E00FE900B53E0FBA3E0FAA3E0F98F828E836A
:1006AE0012278CFF900103E5F0F0A3EFF090010309
:1006BE00E0FCA3E0FD24D1F58274053CF583E090C7
:1006CE0000FFF0A3E4F074D02DF58274053CF583A1
:1006DE00E0FF900100E02FFE9000FFE0340090015B
:1006EE0009F0A3CEF0900109E0FCA3E0FDEC12238B
:1006FE001F900128122913E4FBFA7920784190010A
:10070E0028E0FCA3E0FDA3E0FEA3E0FF1222109080
:10071E00012C12291390012CE0FCA3E0FDA3E0FEB6
:10072E00A3E0FF9007D4122913900101E0FEA3E08D
:10073E00FF7C007D141226D974742FF974083EFACA
:10074E007B0190013B74FFF0A3747BF0A3740AF05D
:10075E0090012CE0FCA3E0FDA3E0FEA3E0FF9001DE
:10076E003E122913123EF6900101E4F0A37406F036
:10077E00E025E0FF900101E033FE900B53E0FBA378
:10078E00E0FAA3E0F98F828E8312278CFF9001038B
:10079E00E5F0F0A3EFF0900103E0FCA3E0FD24D11F
:1007AE00F58274053CF583E09000FFF0A3E4F0744D
:1007BE00D02DF58274053CF583E0FF900100E02F0B
:1007CE00FE9000FFE03400900109F0A3CEF09001FE
:1007DE0009E0FCA3E0FDEC12231F9001281229135F
:1007EE00E4FBFA79207841900128E0FCA3E0FDA318
:1007FE00E0FEA3E0FF12221090012C1229139001AB
:10080E002CE0FCA3E0FDA3E0FEA3E0FF9007D012D6
:10081E002913900101E0FEA3E0FF7C007D14122657
:10082E00D974742FF974083EFA7B0190013B74FF62
:10083E00F0A3747BF0A3740AF090012CE0FCA3E00B
:10084E00FDA3E0FEA3E0FF90013E122913123EF637
:10085E00900101E4F0A37420F0E025E0FF90010187
:10086E00E033FE900B53E0FBA3E0FAA3E0F98F8296
:10087E008E8312278CFF900103E5F0F0A3EFF07446
:10088E00202401FFE433FEEF25E0FFEE338F82F5E7
:10089E008312278CFDACF0900102E025E0FF900161
:1008AE0001E0338F82F58312278CFFC3ED9FFEECA0
:1008BE0095F0900105F0A3CEF0E4A3F0A3F0900123
:1008CE0005E0FEA3E0FFA3E0FCA3E0FDC39FEC9ECA
:1008DE00504D900103E0FEA3E024D0F58274053E56
:1008EE00F583E0FF700F74172DF582E43401F58364
:1008FE00742AF0800C74172DF582E43401F583EF21
:10090E00F0900104E004F07006900103E004F09012
:10091E000108E004F070A7900107E004F0809F90BA
:10092E000105A3E02417F582E43401F583E4F09089
:10093E00013B74FFF0A3747BF0A37412F0900117C7
:10094E00E090013EF0900118E090013FF090011907
:10095E00E0900140F090011AE0900141F090011BEF
:10096E00E0900142F090011CE0900143F07B017A8F
:10097E00097900123EF6900101E4F0A37421F0E033
:10098E0025E0FF900101E033FE900B53E0FBA3E066
:10099E00FAA3E0F98F828E8312278CFF900103E574
:1009AE00F0F0A3EFF074212401FFE433FEEF25E015
:1009BE00FFEE338F82F58312278CFDACF09001028F
:1009CE00E025E0FF900101E0338F82F58312278C42
:1009DE00FFC3ED9FFEEC95F0900105F0A3CEF0E481
:1009EE00A3F0A3F0900105E0FEA3E0FFA3E0FCA3BB
:1009FE00E0FDC39FEC9E504D900103E0FEA3E0246A
:100A0E00D0F58274053EF583E0FF700F74172DF557
:100A1E0082E43401F5837420F0800C74172DF58276
:100A2E00E43401F583EFF0900104E004F0700690D9
:100A3E000103E004F0900108E004F070A7900107B4
:100A4E00E004F0809F900105A3E02417F582E434C2
:100A5E0001F583E4F090013B74FFF0A3747BF0A3E7
:100A6E007421F0A37401F0A37401F0A37417F07B4A
:100A7E00017A097914123EF6900101E4F0A3742272
:100A8E00F0E025E0FF900101E033FE900B53E0FB18
:100A9E00A3E0FAA3E0F98F828E8312278CFF9001D8
:100AAE0003E5F0F0A3EFF074222401FFE433FEEF30
:100ABE0025E0FFEE338F82F58312278CFDACF0908C
:100ACE000102E025E0FF900101E0338F82F58312F1
:100ADE00278CFFC3ED9FFEEC95F0900105F0A3CEA1
:100AEE00F0E4A3F0A3F0900105E0FEA3E0FFA3E085
:100AFE00FCA3E0FDC39FEC9E504D900103E0FEA3CE
:100B0E00E024D0F58274053EF583E0FF700F741774
:100B1E002DF582E43401F5837420F0800C74172DCA
:100B2E00F582E43401F583EFF0900104E004F070F7
:100B3E0006900103E004F0900108E004F070A79025
:100B4E000107E004F0809FED2401FFE43CFEC3EFBB
:100B5E00940EEE94005018900107E475F0011227E0
:100B6E0076FE741725F0F58274013EF583E4F0E409
:100B7E00900125F090013B74FFF0A3747BF0A374F9
:100B8E0021F0A37401F0A37401F0A37417F07B019C
:100B9E007A097928123EF6900101E4F0A37423F04D
:100BAE00E025E0FF900101E033FE900B53E0FBA344
:100BBE00E0FAA3E0F98F828E8312278CFF90010357
:100BCE00E5F0F0A3EFF074232401FFE433FEEF25EC
:100BDE00E0FFEE338F82F58312278CFDACF090018F
:100BEE0002E025E0FF900101E0338F82F5831227AA
:100BFE008CFFC3ED9FFEEC95F0900105F0A3CEF0B7
:100C0E00E4A3F0A3F0900105E0FEA3E0FFA3E0FC57
:100C1E00A3E0FDC39FEC9E504D900103E0FEA3E0C8
:100C2E0024D0F58274053EF583E0FF700F74172D06
:100C3E00F582E43401F5837420F0800C74172DF5E1
:100C4E0082E43401F583EFF0900104E004F07006C5
:100C5E00900103E004F0900108E004F070A7900109
:100C6E0007E004F0809FED2401FFE43CFEC3EF9407
:100C7E000EEE94005018900107E475F001122776DD
:100C8E00FE741725F0F58274013EF583E4F0E490CE
:100C9E000125F090013B74FFF0A3747BF0A3742147
:100CAE00F0A37401F0A37401F0A37417F07B017A22
:100CBE0009793C123EF6900101E4F0A37424F0E0B1
:100CCE0025E0FF900101E033FE900B53E0FBA3E023
:100CDE00FAA3E0F98F828E8312278CFF900103E531
:100CEE00F0F0A3EFF0900103E0FCA3E0FD24D1F5BA
:100CFE008274053CF583E07F00FE9000FFF0A3EFC9
:100D0E00F074D02DF58274053CF583E02FFFE43EA0
:100D1E00FE9000FDF0A3EFF090013B74FFF0A37482
:100D2E007AF0A374EBF0A3EEF0A3EFF07B017A0957
:100D3E007950123EF6900101E4F0A37425F0E025FF
:100D4E00E0FF900101E033FE900B53E0FBA3E0FACD
:100D5E00A3E0F98F828E8312278CFF900103E5F0BA
:100D6E00F0A3EFF0E49000FFF0A3F090097CE070A8
:100D7E0004A3E064016018900103E0FEA3E024D117
:100D8E00F58274053EF583E09000FFF0A3E4F09049
:100D9E000103E0FEA3E024D0F58274053EF583E066
:100DAE00FF900100E02FFF9000FFE03400FE900165
:100DBE0009F0A3EFF0FDAC06EC12231F90012812F0
:100DCE00291390097CE07004A3E06401601EE4FB2B
:100DDE00FA79207841900128E0FCA3E0FDA3E0FE23
:100DEE00A3E0FF12221090012C12291390097CE02F
:100DFE007004A3E064017012900128E0FCA3E0FDF2
:100E0E00A3E0FEA3E0FFA312291390013B74FFF0B1
:100E1E00A3747BF0A3740AF090012CE0FCA3E0FD18
:100E2E00A3E0FEA3E0FF90013E1229137B017A0995
:100E3E007964123EF69000FBE07004A3E064026059
:100E4E00030218A5900101F0A3F0E025E0FF900148
:100E5E0001E033FE900B53E0FBA3E0FAA3E0F98F21
:100E6E00828E8312278CFF900103E5F0F0A3EFF042
:100E7E00E42401FFE433FEEF25E0FFEE338F82F52D
:100E8E008312278CFDACF0900102E025E0FF90016B
:100E9E0001E0338F82F58312278CFFC3ED9FFEECAA
:100EAE0095F0900105F0A3CEF0E4A3F0A3F090012D
:100EBE0005E0FEA3E0FFA3E0FCA3E0FDC39FEC9ED4
:100ECE005055900101E0FEA3E090087475F01412E5
:100EDE002950EE75F014A42583F583E5822DF58255
:100EEE00E5833CF583E0FF900103E0FCA3E024D012
:100EFE00F58274053CF583EFF0900104E004F07088
:100F0E0006900103E004F0900108E004F0709F9059
:100F1E000107E004F08097900101E4F0A304F0E0F3
:100F2E0025E0FF900101E033FE900B53E0FBA3E0C0
:100F3E00FAA3E0F98F828E8312278CFF900103E5CE
:100F4E00F0F0A3EFF0740125E0FFE433FEEF25E0AF
:100F5E00FFEE338F82F58312278CFDACF0900102E9
:100F6E00E025E0FF900101E0338F82F58312278C9C
:100F7E00FFC3ED9FFEEC95F0900105F0A3CEF0E4DB
:100F8E00A3F0A3F0900105E0FEA3E0FFA3E0FCA315
:100F9E00E0FDC39FEC9E5055900101E0FEA3E09052
:100FAE00087475F014122950EE75F014A42583F50B
:100FBE0083E5822DF582E5833CF583E0FF90010306
:100FCE00E0FCA3E024D0F58274053CF583EFF090AD
:100FDE000104E004F07006900103E004F0900108B3
:100FEE00E004F0709F900107E004F08097900101FB
:100FFE00E4F0A37402F0900101E0FCA3E0FD25E013
:10100E00FFEC33FE900B53E0FBA3E0FAA3E0F98F65
:10101E00828E8312278CFF900103E5F0F0A3EFF090
:10102E0090087475F014ED122950EC75F014A42587
:10103E0083F583E0FF7E009000FDEEF0A3EFF090CD
:10104E000103E0FCA3E0FD24D0F58274053CF5839A
:10105E00EFF09000FDE0FF74D12DF58274053CF5A4
:10106E0083EFF0900101E4F0A37403F0900101E02E
:10107E00FCA3E0FD25E0FFEC338F82F58312278C75
:10108E00FF900103E5F0F0A3EFF090097CE070040F
:10109E00A3E064016045ED2401FFE43CFEEF25E092
:1010AE00FFEE33FE900B53E0FBA3E0FAA3E0F98FC3
:1010BE00828E8312278CFDACF0900102E025E0FFBA
:1010CE00900101E0338F82F58312278CFFC3ED9FD1
:1010DE00FEEC95F0900105F0A3CEF0E4900107F040
:1010EE00A3F0900107E0FEA3E0FFD39403EE94007B
:1010FE0040030211B0EF25E0FFEE33FE740B2FF527
:10110E008274013EF583A3E0FD900103E0FAA3E0B3
:10111E0024D0F58274053AF583EDF0900104E004D5
:10112E00F07006900103E004F090097CE07004A3D7
:10113E00E06401601E740B2FF58274013EF583E0AE
:10114E00FF900103E0FCA3E024D0F58274053CF58A
:10115E0083EFF090097CE07004A3E06401600E90D0
:10116E000104E004F07006900103E004F090097CA5
:10117E00E07004A3E064016018900103E0FEA3E0B8
:10118E0024D1F58274053EF583E09000FFF0A3E4D0
:10119E00F0900108E004F07006900107E004F00200
:1011AE0010F0900101E4F0A37404F0900101E0FC52
:1011BE00A3E0FD25E0FFEC33FE900B53E0FBA3E034
:1011CE00FAA3E0F98F828E8312278CFF900103E53C
:1011DE00F0F0A3EFF090087475F014ED122950ECB6
:1011EE0075F014A42583F583E0FF7E007C007D0A54
:1011FE001226D9AC06AD07E412231F90012812293E
:10120E0013900101E0FEA3E090087575F014122909
:10121E0050EE75F014A42583F583E0FF7E007C006C
:10122E007D0A1226D9AC06AD07E412231F90012CBD
:10123E00122913900101E0FEA3E090087675F014D8
:10124E00122950EE75F014A42583F583E0FF7E007D
:10125E007C007D0A1226D9AC06AD07E412231F903E
:10126E000130122913900101E0FEA3E0900877757A
:10127E00F014122950EE75F014A42583F583E0FFC7
:10128E007E007C007D0A1226D9AC06AD07E412233F
:10129E001F900134122913900128E0FCA3E0FDA356
:1012AE00E0FEA3E0FF122358900103E475F0011253
:1012BE002776FC74D025F0F58274053CF583EFF0AB
:1012CE0090012CE0FCA3E0FDA3E0FEA3E0FF1223BF
:1012DE0058900103E475F001122776FC74D025F0C6
:1012EE00F58274053CF583EFF0900130E0FCA3E04D
:1012FE00FDA3E0FEA3E0FF122358900103E475F076
:10130E0001122776FC74D025F0F58274053CF58326
:10131E00EFF0900134E0FCA3E0FDA3E0FEA3E0FFBC
:10132E00122358900103E475F001122776FC74D055
:10133E0025F0F58274053CF583EFF0900101E4F0A1
:10134E00A37405F0900101E0FCA3E0FD25E0FFECA5
:10135E0033FE900B53E0FBA3E0FAA3E0F98F828EED
:10136E008312278CFF900103E5F0F0A3EFF09008B5
:10137E007475F014ED122950EC75F014A42583F554
:10138E0083E0FCE4122324900128122913E4FBFAD3
:10139E0079207841900128E0FCA3E0FDA3E0FEA3B4
:1013AE00E0FF122210E4FBFA79C8784212210712EC
:1013BE002358900109EEF0A3EFF0900109E0FEA38F
:1013CE00E0FD900103E0FAA3E0FB24D0F582740562
:1013DE003AF583EDF0EEFF74D12BF58274053AF5F4
:1013EE0083EFF0900101E4F0A37406F0900101E0A8
:1013FE00FCA3E0FD25E0FFEC33FE900B53E0FBA3D6
:10140E00E0FAA3E0F98F828E8312278CFF900103FE
:10141E00E5F0F0A3EFF090087475F014ED1229507A
:10142E00EC75F014A42583F583E0FCE412232490DC
:10143E000128122913E4FBFA79207841900128E063
:10144E00FCA3E0FDA3E0FEA3E0FF122210E4FBFAF2
:10145E0079C87842122107122358900109EEF0A3A1
:10146E00EFF0900109E0FEA3E0FD900103E0FAA386
:10147E00E0FB24D0F58274053AF583EDF0EEFF74AF
:10148E00D12BF58274053AF583EFF0900101E4F06B
:10149E00A37420F0E025E0FF900101E033FE900BF5
:1014AE0053E0FBA3E0FAA3E0F98F828E8312278C20
:1014BE00FF900103E5F0F0A3EFF074202401FFE4A8
:1014CE0033FEEF25E0FFEE338F82F58312278CFD7E
:1014DE00ACF0900102E025E0FF900101E0338F8235
:1014EE00F58312278CFFC3ED9FFEEC95F09001055E
:1014FE00F0A3CEF0E4A3F0A3F0900105E0FEA3E08C
:10150E00FFA3E0FCA3E0FDC39FEC9E503C74002DB6
:10151E00F58274093CF583E0FF900103E0FCA3E043
:10152E0024D0F58274053CF583EFF0900104E004BD
:10153E00F07006900103E004F0900108E004F070F2
:10154E00B8900107E004F080B0900101E4F0A374BC
:10155E0021F0E025E0FF900101E033FE900B53E017
:10156E00FBA3E0FAA3E0F98F828E8312278CFF9003
:10157E000103E5F0F0A3EFF074212401FFE433FE44
:10158E00EF25E0FFEE338F82F58312278CFDACF052
:10159E00900102E025E0FF900101E0338F82F58398
:1015AE0012278CFFC3ED9FFEEC95F0900105F0A382
:1015BE00CEF0E4A3F0A3F0900105E0FEA3E0FFA3BC
:1015CE00E0FCA3E0FDC39FEC9E503C74142DF5820D
:1015DE0074093CF583E0FF900103E0FCA3E024D006
:1015EE00F58274053CF583EFF0900104E004F07091
:1015FE0006900103E004F0900108E004F070B8904A
:10160E000107E004F080B0900101E4F0A37422F031
:10161E00E025E0FF900101E033FE900B53E0FBA3C9
:10162E00E0FAA3E0F98F828E8312278CFF900103DC
:10163E00E5F0F0A3EFF074222401FFE433FEEF2572
:10164E00E0FFEE338F82F58312278CFDACF0900114
:10165E0002E025E0FF900101E0338F82F58312272F
:10166E008CFFC3ED9FFEEC95F0900105F0A3CEF03C
:10167E00E4A3F0A3F0900105E0FEA3E0FFA3E0FCDD
:10168E00A3E0FDC39FEC9E503C74282DF582740997
:10169E003CF583E0FF900103E0FCA3E024D0F5824B
:1016AE0074053CF583EFF0900104E004F0700690B1
:1016BE000103E004F0900108E004F070B890010717
:1016CE00E004F080B0900101E4F0A37423F0E02573
:1016DE00E0FF900101E033FE900B53E0FBA3E0FA34
:1016EE00A3E0F98F828E8312278CFF900103E5F021
:1016FE00F0A3EFF074232401FFE433FEEF25E0FFA7
:10170E00EE338F82F58312278CFDACF0900102E050
:10171E0025E0FF900101E0338F82F58312278CFFC5
:10172E00C3ED9FFEEC95F0900105F0A3CEF0E4A37F
:10173E00F0A3F0900105E0FEA3E0FFA3E0FCA3E020
:10174E00FDC39FEC9E503C743C2DF58274093CF514
:10175E0083E0FF900103E0FCA3E024D0F582740542
:10176E003CF583EFF0900104E004F0700690010365
:10177E00E004F0900108E004F070B8900107E00476
:10178E00F080B0900101E4F0A37424F0E025E0FFB6
:10179E00900101E033FE900B53E0FBA3E0FAA3E0CF
:1017AE00F98F828E8312278CFF900103E5F0F0A350
:1017BE00EFF0900950E0FCE4122324900128122946
:1017CE0013900128E0FCA3E0FDA3E0FEA3E0FF12CE
:1017DE0023589000FFEEF0A3EFF09000FFE0FCA383
:1017EE00E0FDECFF900103E0FAA3E0FB24D1F582CB
:1017FE0074053AF583EFF074D02BF58274053AF543
:10180E0083EDF0900101E4F0A37425F0E025E0FFF4
:10181E00900101E033FE900B53E0FBA3E0FAA3E04E
:10182E00F98F828E8312278CFF900103E5F0F0A3CF
:10183E00EFF0900964E0FCE41223249001281229B1
:10184E0013E4FBFA79207841900128E0FCA3E0FD37
:10185E00A3E0FEA3E0FF122210E4FBFA79C878425F
:10186E001221071223589000FFEEF0A3EFF0900024
:10187E00FFE0FEA3E0FD900103E0FAA3E0FB24D01D
:10188E00F58274053AF583EDF0EEFF74D12BF582F7
:07189E0074053AF583EFF039
:0118A5002220
:0400030075AE0122B3
:0400070075A67E223A
:041FF00075A60122AF
:0F200000E4F5F5907FE27492F0000002000022F8
:10397F0063CF0DDE4F4B0000000000000000000081
:10398F000000000000000000000000000041637410
:10399F007561746F725F446574656374696F6E5F90
:1039AF004661696C00004D6F746F725F4A616D0004
:1039BF0000000000000000000000000000000041B7
:1039CF0063747561746F725F4A616D5F54656D707A
:1039DF006F72617279000000426C6F636B5F6E757E
:1039EF006D6265725F73657175656E63650000006A
:1039FF0000416E74656E6E61204275737900000030
:103A0F0000000000000000000000436865636B7356
:103A1F00756D5F6572726F7200000000000000002C
:103A2F0000000050726F6365647572655F53657156
:103A3F0075656E63655F6572726F72004461746164
:103A4F005F6572726F7200000000000000000000DE
:103A5F0000000000004465766963655F4469736127
:103A6F00626C656400000000000000000000456506
:103A7F0070726F6D5F4572726F7200000000000010
:103A8F0000000000000000416E74656E6E612046FC
:103A9F0061696C6564000000000000000000000018
:103AAF00466C6173685F65726173655F6572726F93
:103ABF00720000000000000000466C6173685F65D3
:103ACF0072726F7200000000000000000000000022
:103ADF0000004E6F745F43616C696272617465645C
:103AEF0000000000000000000000004E6F745F43F4
:103AFF006F6E6669677572656400000000000000F4
:103B0F000000000048617264776172655F657272D0
:103B1F006F720000000000000000000000536F668D
:103B2F0074776172655F6572726F720000000000DA
:103B3F000000000000004F75745F6F665F52616E8A
:103B4F00676500000000000000000000000000504A
:103B5F006F736974696F6E5F4C6F73740000000050
:103B6F00000000000000000052616D5F6572726F0F
:103B7F0072000000000000000000000000000000C4
:103B8F00005365676D656E745F4E756D6265725F2C
:103B9F0053657175656E63650000554152545F65DD
:103BAF0072726F7200000000000000000000000041
:103BBF00000000556E6B6E6F776E5F70726F63658E
:103BCF00647572650000000000000000544D415FF5
:103BDF00416C61726D5F6D696E6F72000000000065
:103BEF000000000000544D415F416C61726D5F6DCC
:103BFF00616A6F7200000000000000000000476162
:103C0F00696E5F6F75745F6F665F52616E67650097
:103C1F0000000000000000526561645F4F6E6C7918
:103C2F000000000000000000000000000000000085
:103C3F00556E6B6E6F776E5F506172616D657465F7
:103C4F00720000000000000000556E6B6E6F776E03
:103C5F005F4465766963655F4E756D6265720000DE
:103C6F000000576F726B696E675F736F6674776171
:103C7F0072655F6D697373696E6700496E76616C0B
:103C8F0069645F46696C655F436F6E74656E74003F
:103C9F0000000000446F776E6C6F61645F696E5F48
:103CAF0070726F67726573730000000000466F7269
:103CBF006D61745F6572726F72000000000000002A
:103CCF00000000000000556E737570706F727465A0
:103CDF00645F50726F636564757265000000004920
:103CEF006E76616C69645F53657175656E636500AF
:103CFF0000000000000000004163747561746F7272
:103D0F005F496E746572666572656E63650000006B
:103D1F000000000000000000000000000000000094
:103D2F000000000000000000000000000000000084
:103D3F000000000000000000000000000000000074
:033D4F0000000071
:10775200900B6EE0FCA3E0FDA3E0FEA3E0FFE412C9
:10776200231A7B8A7A3D79167846122210E4FBFAB4
:10777200F97842122210A804A905AA06AB07E4FF71
:10778200FE7D807C47122012122358AD07AC06EC16
:10779200F5CBAF058FCA75C834759850C2B2C2987E
:0F77A200C299E4F5A8D2AFD2ABD2A9C2ACD2BC87
:0177B10022B5
:10716D00900135EBF0A3EAF0A3E9F0A3ECF0A3ED69
:01717D00F021
:10717E00A3E0FFA3E0A3CFF0A3EFF0E4A3F0A3F00E
:10718E00900138E0FEA3E0FF90013EE06E7003A395
:10719E00E06F6065900135E0FBA3E0FAA3E0F990A3
:1071AE00013EE0FEA3E0F5828E8312269AFF900147
:1071BE003CE0F0A3E06FF0E4FD90013CE0FEA3E0C4
:1071CE00FF5401FCEEC313FEEF13FF90013CEEF0F3
:1071DE00A3EFF0AF04EF600C90013CE06484F0A3E9
:1071EE00E06408F00DEDB408D090013FE004F070BB
:1071FE008F90013EE004F0808790013CE0FEA3E01A
:01720E00FF80
:01720F00225C
:0A000E00C2998F993099FDC2992222
:1076F100D2B2E4F517901545E0FCA3E0FDD3951750
:10770100EC94004049901547E0FAA3E02517F58273
:10771100E43AF583E0F516B47E1DE5176019ED2412
:10772100FFFFEC34FFFEEF65177001EE60097F7D0E
:1077310012000E7F5E8010E516B47D097F7D120078
:107741000E7F5D8002AF1612000E051780A7C2B230
:017751002215
:104E36007F017E0012786D9015477412F0A374E11D
:104E4600F0E490140FF0A3F0901545F0A3F090094C
:104E56007CE0FEA3E0FF64014E700690013274040C
:104E6600F0EF64024E70069001327403F090154321
:104E7600E0FEA3E0FF64BF4E7012900132E0FD90A9
:104E86001548E02DF0901547E03400F0901547E006
:104E9600FCA3E0FDF5828C83C083C082901545E4B7
:104EA60075F001122776FAD082D083E58225F0F5D7
:104EB60082E5833AF583747EF09011AFA3E0FB8D13
:104EC600828C83C083C082901545E475F001122759
:104ED60076FCD082D083E58225F0F582E5833CF529
:104EE60083EBF0901547E0FAA3E0F5828A83C0834E
:104EF600C082901545E475F001122776FAD082D06B
:104F060083E58225F0F582E5833AF583EFF030E01C
:104F16000F901543E07004A3E064BF600302500DD8
:104F2600901543E07004A3E064BF7003024FF9904C
:104F3600097CE07004A3E06401702C901547E0FE44
:104F4600A3E0F5828E83C083C082901545E475F098
:104F560001122776FED082D083E58225F0F582E520
:104F6600833EF5837401F09011B3A3E0FF901547DB
:104F7600E0FCA3E0FDF5828C83C083C082901545DA
:104F8600E475F001122776FAD082D083E58225F007
:104F9600F582E5833AF583EFF0901413A3E0FF8DD5
:104FA600828C83C083C082901545E475F001122778
:104FB60076FCD082D083E58225F0F582E5833CF548
:104FC60083EFF0901413E0FF901547E0FCA3E0F5A3
:104FD600828C83C083C082901545E475F001122748
:104FE60076FCD082D083E58225F0F582E5833CF518
:104FF60083EFF0901413E0FEA3E0FF901546E02F38
:10500600F0901545E03EF0901547E0FEA3E0FFF571
:10501600828E83C083C082901545E475F001122705
:1050260076FCD082D083E58225F0F582E5833CF5D7
:1050360083E4F08F828E83C083C08290154575F01D
:1050460001122776FED082D083E58225F0F582E52F
:10505600833EF583E4F0901547E0FEA3E0FFF5827A
:105066008E83C083C082901545E475F001122776C1
:10507600FCD082D083E58225F0F582E5833CF5837A
:10508600747EF0EF2401FFE43EFAA9077B01901538
:1050960046E024FCFD901545E034FFFC74FF9001CA
:1050A6003AF0A3F012716D900133EEF0A3EFF0F435
:1050B600FFEEF4900133F0A3EFF0901545E0FCA36A
:1050C600E0FD901547E0FAA3E0FB2DF582EA3CF5FA
:1050D60083E58224FDF582E58334FFF583EFF090C6
:1050E6000133E0FFEB2DF582EA3CF583E58224FEF1
:0D50F600F582E58334FFF583EFF01276F1CB
:015103002289
:1053BD00E490140DF0A3F09011B1F0A3F09014113E
:1053CD00F0A3F09015477411F0A374B5F0126DDAD7
:1053DD0090140DEEF0A3EFF04E60030256479015BA
:1053ED0045E0FEA3E0FF901547E0FCA3E0FD2FF59F
:1053FD0082EC3EF583E58224FEF582E58334FFF5EC
:10540D0083E0F4FF901545E0FAA3E0FBED2BF58268
:10541D00EC3AF583E58224FEF582E58334FFF583CE
:10542D00EFF0901545E0FEA3E0FF901547E0FAA3DD
:10543D00E0FB2FF582EA3EF583E58224FDF582E55A
:10544D008334FFF583E0F4FF901545E0FCA3E0FD08
:10545D00EB2DF582EA3CF583E58224FDF582E583AB
:10546D0034FFF583EFF0901548E02401FF901547C8
:10547D00E03400FAA9077B01ED24FEFDEC34FFFCBE
:10548D0074FF90013AF0A3F012716DEF4E600A9027
:10549D00140EE04404F0025647901547E0FEA3E0D9
:1054AD00F5828E83C083C082901411E475F00112D1
:1054BD002776FED082D083E58225F0F582E5833E06
:1054CD00F583E0647E600A90140EE04408F0025605
:1054DD0047901547E0FEA3E0FFF5828E83C083C0A1
:1054ED0082901411E475F001122776FCD082D083DE
:1054FD00E58225F0F582E5833CF583E0FD9011AD65
:10550D00E4F0A3EDF08F828E83C083C082901411DE
:10551D00E475F001122776FED082D083E58225F066
:10552D00F582E5833EF583E0FF901541E4F0A3EFAE
:10553D00F0901412E02403FF901411E03400FEC328
:10554D00901546E09FFF901545E09EFE901542E0B8
:10555D0030E00302562890097CE07004A3E064015A
:10556D00702E901547E0FCA3E0F5828C83C083C0BC
:10557D0082901411E475F001122776FCD082D0834D
:10558D00E58225F0F582E5833CF583E0900132F06C
:10559D00901547E0FEA3E0FFF5828E83C083C082A5
:1055AD00901411E475F001122776FCD082D083E5BA
:1055BD008225F0F582E5833CF583E0FD9011B1E4A1
:1055CD00F0A3EDF08F828E83C083C082901411E41E
:1055DD0075F001122776FED082D083E58225F0F595
:1055ED0082E5833EF583E0FD901547E0FEA3E0F5EF
:1055FD00828E83C083C082901411E475F00112274E
:10560D0076FED082D083E58225F0F582E5833EF5E6
:10561D0083E0FE7C00E42DFFEC3EFE901411E0FCD7
:10562D00A3E024B5F58274113CAD8290154AF0A328
:10563D00EDF0901411EEF0A3EFF090140DE0FEA339
:02564D00E0FF7C
:01564F002238
:106DDA00C2B2E490140DF0A3F0900134F09001A037
:106DEA00F0A3F0127B932009057E007F01223098E0
:106DFA00F5C298900133E599F0127B93900133E044
:106E0A00FF647D7003026E99A3E0B40138EFB45DAC
:106E1A0006900133747DF0900133E0B45E03747E12
:106E2A00F0900133E0FF9001A0E475F0011227769B
:106E3A00FC74B525F0F58274113CF583EFF0E4900B
:106E4A000134F080A1900133E0FF9001A0E475F0D5
:106E5A0001122776FC74B525F0F58274113CF5838E
:106E6A00EFF0647E70809001A0E0FEA3E0FFD3946F
:106E7A0001EE94005003026DF0901545EEF0A3EF79
:106E8A00F0E4900134F09001A0F0A3F0FEFF22900C
:086E9A0001347401F0026DF0F7
:1061BC005E0000000000000000000000287C287C2D
:1061CC00280000000000000000000000000000009B
:1061DC0000000000060000000000000000000000AD
:1061EC0000000000000028102800000010381000EB
:1061FC0000002060000000000808080000004000BB
:10620C00000000006030180C00003C524A3C0000BA
:10621C00447E4000000064524A44000024424A3448
:10622C0000001C107E1000004E4A4A3200003C4A0E
:10623C004A30000002720A060000344A4A34000058
:10624C000C52523C00006C0000000000167600005E
:10625C0000001028440000002828000000004428FA
:10626C00100000000402B2120C000000000000003C
:10627C007C12127C00007E4A4A3400003C424242AE
:10628C0000007E42423C00007E4A4A4200007E0AE8
:10629C000A0200003C42427200007E08087E0000A8
:1062AC00427E4200000020423E0200007E18244242
:1062BC0000007E40404000007E0408047E007E18F2
:1062CC00307E00003C42423C00007E12120C00006A
:1062DC007E42627E00007E12324C0000444A4A32FA
:1062EC000000027E020000003E40403E00001E20E6
:1062FC0040201E007E2010207E00760808760000CC
:10630C0006087806000062524A46000000000000B1
:10631C000000000000000000000000000000000071
:10632C00000000004040400000007E7E7E7E7E7EAD
:103D52005700DF415247555320544543484E4F4C7C
:103D62004F4749455300000000005700C84E4F20FE
:103D720044455649434520464F554E4400000000F5
:103D8200000000006064000000000000000000006D
:103D9200000000C0B088848381818181818181811A
:103DA2008181838488B0C000000000000000000010
:103DB20000FF80BFA0A0A0A0BF80FF000000000005
:103DC20000000000000000000000000000000000F1
:103DD200FF000000000000000000000000000000E2
:103DE20000000000000000000000000060640064A9
:103DF200000000000000000000000000000000FFC2
:103E0200017D4545454545457D01FF002070A820BF
:103E12002020202020A8702000FF01BDA5A5A5A577
:103E2200BD01FF002070A8202020202020A87020A3
:103E32000001020408102040FF4020100804020183
:103E42000000000000000000000000000000000070
:043E5200000000006C
:0F7A6D0024B8907F05F07F967E00127A7CE4F0BB
:107A7C00EF64964E7008D2B6D2B7C2B6C2B7D3EF87
:107A8C009431EE94005004D2B6C2B6C3EF9432EEE9
:107A9C009400400DD3EF9464EE94005004D2B7C21E
:027AAC00B722FF
:107C8E00E4FDFCEF127A6DD2B4D3ED9431EC940096
:107C9E005012E4907F05F07F96FE127A7C0DBD00A7
:067CAE00010C80E5C2B4E8
:017CB40022AD
:1075B200E4907F03F0907F0774FFF0E4907F09F07E
:1075C200907F05F0907F0D74FFF0D2C4C2C5C2B4A3
:1075D200C2B5C2B6C2B7D2C3907F057460F07F96BF
:1075E2007E00127A7C74A0F0127A7C74A9F0127A6E
:1075F2007C74A4F0127A7C74B8F0127A7774AFF0CB
:10760200127A7CE4FF127C8E7F01127C8E7F021242
:107612007C8E7F03127C8E7C007DDFE4FF125ADBBE
:017622002245
:065ADB00AB05AA04AD07B3
:105AE100E4F516F517F518F519F51CF51DED127A03
:105AF1006DAF05127C8EE4907F05F07F96FE127AE1
:105B01007CD2B4D3E5179419E51694004003025CE6
:105B11009CEB2517F582EA3516F583E06420703693
:105B21000517E51770020516900564E0907F057072
:105B310003F0800374FFF0AF1DAE1C127A7C051DCB
:105B4100E51D7002051CFFAE1C127A7C051DE51DCA
:105B510070BF051C80BBEB2517F582EA3516F5836E
:105B6100E07003C2B422EB2517F582EA3516F583FE
:105B7100E0C39461402CEB2517F582EA3516F583D5
:105B8100E0D3947A501CEB2517F582EA3516F5839C
:105B9100E0F51E24E0FFEB2517F582EA3516F583C3
:105BA100EFF0EB2517F582EA3516F583E0D3941F64
:105BB1004010EB2517F582EA3516F583E0C39460B2
:105BC100400DEB2517F582EA3516F5837421F0EBCC
:105BD1002517F582EA3516F583E024DFF51BE43459
:105BE100FFF51AD3E5199405E518940050799061F1
:105BF100BC75F006E51B122950E51A75F006A425BF
:105C010083F583E5822519F582E5833518F583E46B
:105C110093FF7007F5187519058041900564E0B48C
:105C21000104EFF480239061BC75F006E51B122995
:105C310050E51A75F006A42583F583E5822519F54B
:105C410082E5833518F583E493907F05F0AF1DAEAF
:105C51001C127A7C051DE51D7002051C0519E5194C
:105C610070020518025BE4900564E0FF7004907F08
:105C710005F0EFB40106907F0574FFF0AF1DAE1C77
:105C8100127A7C051DE51D7002051CE4F518F51955
:0B5C91000517E51770020516025B0402
:015C9C0022E5
:1073DF00E4FF127C8E7F03127C8EC2B4C2B5C2B69C
:1073EF00C2B7907F0574AFF07F967E00127A7C74DF
:1073FF00B9F0127A77D2B4E4FD74642DF582E434D7
:10740F0000F583E0907F05F0EDFF7E00127A7C0D92
:10741F00EDB464E5C2B4C2B5C2B6C2B7907F05740D
:10742F00BA127A72D2B4E4FD74002DF582E43400FE
:10743F00F583E0907F05F0EDFF7E00127A7C0DED75
:05744F00B464E5C2B4C5
:017454002215
:107D2800E4F9E975F019A42469F582E43405AD8213
:0B7D3800FCAF01125ADB09E9B404E7BC
:017D4300221D
:107BC800EE7030EF14601114601514601914601D04
:107BD8002404701FC2C08002D2C0C2C1C2C222C265
:107BE800C0D2C1C2C222C2C0C2C1D2C222D2C0D275
:047BF800C1D2C22212
:10001E00907FE2E04480F0907FB07438F0907FB42F
:04002E007470F022D8
:101F3C0012011001000000088304000000010102DE
:101F4C00000109092100010001222E0009022200D2
:101F5C00010100C0FA09040000010300000009217E
:101F6C0000010001222E00070581030800642E06E3
:101F7C00A0FF09A5A10109A609A51580257F750853
:101F8C009540B10209A71580257F75089508810237
:101F9C0009A91580257F750895409102C004030995
:101FAC000426034100720067007500730020005482
:101FBC00006500630068006E006F006C006F0067C6
:101FCC00006900650073001403430054005800447A
:101FDC00002D00330030002D005200FF1FA9FF1F01
:041FEC00ADFF1FD353
:1074CA00900193E4F0A3F0A3F0900189F0A3F07F78
:1074DA000AFEFDFC900B6EE0F8A3E0F9A3E0FAA324
:1074EA00E0FB1227C4E47B02FAF9F812284F7B80EA
:1074FA007A8D795B780012284FEF2405FFE43EFE6F
:10750A00E43DFDE43CFCE47B0AFAF9F812284FEF6B
:10751A0014F5E175EA3875EA1875EC0C75EB2875FF
:10752A00E6BA75E6BE75EB2275E9BF75EE80E4F53D
:05753A00E843A7012257
:041FF40043EA40225A
:041FF80075EAB022B4
:107D440090018DE0D39400782340077604121FFC41
:087D54008002760375EAB022FB
:106EA200900193E0FBA3E0FAA3E0F9EA494B7003F7
:106EB200026F64900189E0FEA3E0FF4E700DE5EAE7
:106EC200648054804430F5EA026F5890016BEEF012
:106ED200A3EFF0D39408EE64809480400990016B94
:106EE200E4F0A37408F0E5EA648054804430FF9033
:106EF200016BA3E04FF5EAE4FFFED390016CE09F43
:106F0200EE6480F890016BE0648098401C900193DD
:106F1200E0FBA3E475F001122776A9F0FA122681AC
:106F2200F5E70FBF00010E80D190016BE0FEA3E0F8
:106F3200FFC390018AE09FFD900189E09EFCF0A3CF
:106F4200EDF04C701A900188E0600BC3EF9408EEEC
:106F5200648094805009900193E4F0A3F0A3F07F41
:076F6200012275EA907F0097
:016F69002205
:10799F00900173EBF0A3EAF0A3E9F0D3ED9408ECB8
:1079AF006480948040047C007D08E5EA6480548004
:1079BF0044304DF5EAED1DAE0470011C4E6017907A
:1079CF000173E0FBA3E475F001122776A9F0FA1218
:0779DF002681F5E780DF229D
:106A520090018EE024FE602A14603A24E2606314FE
:106A6200607524216003026AF790019374FFF0A31A
:106A7200741FF0A3743CF0900189E4F0A37412F047
:106A8200807790019374FFF0A3741FF0A37458F001
:106A9200901F5A803E90018DE075F003A424E7F523
:106AA20082E5F0341FF583E493FB740193FA7402D8
:106AB20093F9900193EBF0A3EAF0A3E9F012268197
:106AC200802890019374FFF0A3741FF0A3744FF019
:106AD200901F4EE493801390019374FFF0A3741FF0
:106AE200F0A3747BF0901F7AE493FF900189E4F0A5
:106AF200A3EFF0800443EA4022900192E0FE90016D
:106B020091E0FDEDFF900189E0FCA3E0FDC39FEE63
:106B12006480F8EC64809850047B0180027B0090D2
:106B22000188EBF0D3ED9FEE6480F8EC648098402E
:0D6B320006A3EEF0A3EFF053EA7F126EA26F
:016B3F002233
:1079E60090016B7401F0A37401F0A3748BF0E5EDC4
:1079F600540F6408600643EA407F0022E4FFFE90CD
:107A0600016BE0FBA3E475F001122776A9F0FAE515
:107A1600EF1226C70FBF00010EEF64084E70E04359
:047A2600ED807F016F
:017A2A002239
:107B5D00900193E4F0A3F0A3F0900189F0A3F0A3BA
:107B6D00E05460701DA3E024FB600E14600E24FD34
:107B7D00600D2408700C021FF4021FF8026A5202F5
:067B8D007D4443EA4022A2
:107D0200126EA2EF701F90018CE0B40512A3E0FF87
:107D12004480F5EEEF7823600476038002760290C9
:067D2200018C74FFF02249
:103E560042167F0000421707000041187E004116F7
:103E66007E0041187C00411551004118C1004117E0
:103E76000400411550004117090041170A00411678
:0A3E8600C3004118C00041154E00B2
:0B78BC009000F7EBF0A3EAF0A3E9F066
:1078C700E4A3F0D2B2F0901708E024FFFF90170767
:1078D700E034FFFE9000FAE0D39FE49E5021900031
:1078E700F7E0FBA3E0FAA3E0F9A3E0F582758300D4
:1078F70012269AFF12000E9000FAE004F080C7C229
:01790700B2CD
:01790800225C
:1070C4009000F7EEF0A3EFF0A3ECF0A3EDF0A3EA49
:0470D400F0A3EBF04A
:1070D800A3E0907FE0F09000FEE0FFC39410502200
:1070E800EF7007A37480F0A3E4F0EFB401099000F7
:1070F800FF74C0F0A3E4F09000FFE0FEA3E0FF12ED
:1071080077B2E4F50AF50B9000FCE024FFFF90004D
:10711800FBE034FFFED3E50B9FE50A9E504090004C
:10712800FAE0250BFE9000F9E0350A9000FFF0A385
:10713800CEF09000F7E0FCA3E0250BF582EC350AD1
:10714800F583E0F5089000FFE0FEA3E0FFAD08122C
:10715800753F8F09050BE50B70AD050A80A9907F77
:04716800E07401F0DE
:01716C002200
:0665DE00907FE07401F063
:1065E40090167EE0D3942C748094814002E4F09061
:1065F400167EE0FF04F074522FF582E43415F5831F
:10660400747EF090167EE07E002452F9EE3415FA82
:106614007B0190154FE0FF90167EE0FE04F074526B
:106624002EF582E43415F583EFF0901706E0FF9021
:10663400167EE0FE04F074522EF582E43415F583E0
:10664400EFF09018C0E0FF90167EE0FE04F0745264
:106654002EF582E43415F583EFF090167EE0FF0406
:10666400F074522FF582E43415F5837401F090161A
:106674007EE0FF04F074522FF582E43415F583E4D0
:10668400F090167EE0FF04F074522FF582E4341586
:10669400F583E4F090167EE0FF04F074522FF58247
:1066A400E43415F583E4F090167EE0FF04F07452B0
:1066B4002FF582E43415F583E4F090167EE0FF04B0
:1066C400F074522FF582E43415F583747EF074FF70
:1066D40090013AF0A3F07D067C0012716DEFF4FF97
:1066E400EEF4FE90167EE0FC244FF582E43415F5BA
:1066F40083EFF0EEFF74502CF582E43415F583EF4C
:10670400F0E4901704F090170A04F0E4901709F0ED
:016714002262
:107AAE0043EB287F087E00E4FDFCC3ED9FEE64806F
:107ABE00F8EC648098500AE4F5E60DBD00010C80E8
:107ACE00E97D01E5EB648054804420FBED64027097
:0C7ADE00047D4080027D00EB4D4FF5EB75
:017AEA002279
:107B24007E007F407D007B017A1679C4122A8B7E09
:107B3400007F407D007B017A167981122A8B901890
:107B4400397440F090187FF075AE551274CA120063
:097B54001EE490167EF0027AAEE8
:10601A00E49000F6F090187DE0B40116901551E076
:10602A007010FFFE127BC81273DF9015517401F0D5
:10603A00C2C39018C1E0640160030261379018C0BE
:10604A00E0FF700302611FB4E02BE4907FE0F09060
:10605A00183A7480F0A3E4F0FF7E801277B29018A9
:10606A003A74C0F0A3E4F0FF7EC01277B21265DE84
:10607A00E49018C0F09018C0E064EB7066901713B3
:10608A00E0FF9016C1E4F0A3EFF0901716E0704B12
:10609A00901714E0FF9018C2F0901715E09018C3FB
:1060AA00F0FDEFFE7C00E42DFFEC3E90170BF0A311
:1060BA00EFF07E177F1790170BE0FCA3E02400F5A2
:1060CA008274803CAD82FC9016C1E0FAA3E0FBE446
:1060DA009000FDF0A37410F01270C41265E4E4900D
:1060EA0018C0F09018C0E064ED7039901713E0649E
:1060FA00417031A3E0B4522CE4907FE0F07D017F3F
:10610A00FD7EFF12753F1265DEE49018C0F090160E
:10611A00C304F0800F7B017A17790D1278BC9017AF
:10612A00047401F0E4901550F09018C1F030984BC7
:10613A00C2989000F6E599F090167EE0D3942C74FC
:10614A008094814002E4F09000F6E0FF90167EE031
:10615A00FE04F074522EF582E43415F583EFF0EF65
:10616A00B47E1890167EE0D39401400FE490170491
:10617A00F090170A04F0E4901709F0C3901680E033
:10618A00943090167FE09475400DE4F0A3F09018D7
:10619A007DF0121FF080FE901680E004F0700690E9
:1061AA00167FE004F09016C3E0B40105121FF080D8
:0161BA00FEE6
:0161BB0022C1
:107BFC00900170EBF0A3EAF0A3E9F0ED1DAE047078
:107C0C00011C4E601C900170E0FBA3E475F00112A6
:107C1C002776A9F0FA122681FF9016C9E02FF08082
:027C2C00DA225A
:041FFC0053EADF22A3
:10510400E490016BF0A3F090016EF090183CE06025
:10511400030253BC901681E024FD60030253BC904B
:105124001839E0F97069EFD3940150030253BCEFCE
:1051340024FFFBE434FFFA901685E0F8A3E0F5823F
:105144008883C39BE5839A5004AB828004EF24FFD9
:10515400FB90016BEBF0E904FD901685A3E0900150
:105164006DF0743C2DF582E43418F583E0FB7A008D
:10517400743D2DF582E43418F583E0F582758300DF
:10518400FEE42BFFEA3E901707F0A3EFF08023EF35
:10519400FB901685E0F8A3E0F5828883C39BE58342
:1051A40094005004AF82800090016BEFF0901839A6
:1051B400E0FD743C2DF9E43418FA7B0190016BE0B6
:1051C400FD7C00127BFC90016BE0FF7E0090168456
:1051D400E02FF0901683E03EF0C3901686E09FFF28
:1051E400901685E09EFEF0A3EFF04E60030253BCE0
:1051F400901681F0901841E0540190016FF09018DE
:1052040042E0FF64E0600DEF64EB6008EF64ED6082
:10521400030252F3E4F990016CF090016DE014FF85
:1052240090016CE0FED39F4003025332743F2EF58D
:1052340082E43418F583E0FF647D70030252E49045
:10524400016EE064017070EFB45D2C90154EE0FFC8
:10525400E92FFFE433FE740D2FF58274173EF583B6
:10526400747DF009901708E024FFF0901707E034EC
:10527400FFF0E490016EF090016CE0243FF582E4CD
:105284003418F583E0645E705D90154EE0FFE92FFD
:10529400FFE433FE740D2FF58274173EF583747E9C
:1052A400F009901708E024FFF0901707E034FFF0AE
:1052B400E490016EF0802F90016CE0243FF582E4CD
:1052C4003418F583E0FF90154EE0FDE92DFDE4333D
:1052D400FC740D2DF58274173CF583EFF0098006FC
:1052E40090016E7401F090016CE004F002521EE42F
:1052F40090016CF090016DE014FF90016CE0D39F7D
:10530400502CE0FF243FF582E43418F583E0FE904E
:10531400154EE0FDEF2DFDE433FC740D2DF5827484
:10532400173CF583EEF090016CE004F080C6901514
:105334004EE0243DF0E0FFD3901708E09F9017075C
:10534400E094005073E49018C0F090016FE070593D
:10535400901842E0FFB4E018901840E090154FF028
:10536400901841E0901706F09018C074E0F080396E
:10537400EFB4EB18901840E090154FF0901841E00E
:10538400901706F09018C074EBF0801D901842E05E
:10539400B4ED16901840E090154FF0901841E0904D
:1053A4001706F09018C074EDF090187C7401F0E4C6
:0853B40090016DF090154EF020
:0153BC0022CE
:107A2B0090183CE0603BB405089017057401F0809A
:107A3B002278817C167D017B017A18793C7E007F50
:107A4B004012265B7E007F407D007B017A1679C455
:107A5B00122A8B90183CE0147007E4F5AE90168157
:027A6B00F02207
:10701A00E4FFFE90018BE0FBB4210CA3E0B4090766
:10702A00E4901839F00F22EB64A160030270C1905A
:10703A00018CE0640160030270C190167EE0FF7C5F
:10704A0000E490016BF0A3EFF0A3E4F0901550E098
:10705A00FF2452F582E43415F583E090016EF07452
:10706A00532FF582E43415F583E090016FF0901503
:10707A0050E02454F582E43415F583E0900170F071
:10708A0074552FF582E43415F583E0900171F09080
:10709A001550E02456F582E43415F583E090017228
:1070AA00F053EA7F7B017A01796B7D0812799FE4BC
:0970BA0090187FF07F01227F0095
:0170C30022AA
:03003300025C9DCF
:105C9D00C0E0C0F0C083C082C0D075D000C000C0CD
:0D5CAD0001C002C003C004C005C006C0074E
:105CBA00900168E4F0A3F0A3F090167FF0A3F090AF
:105CCA00187D04F0E5E830E111E5EA30E609E5ED92
:105CDA005430600353EABF53E8FDE5E830E44F432C
:105CEA00EA3853EADF90187FE0FFC3943850397ED0
:105CFA000074572FF9EE3415FA7B01901550E029FC
:105D0A00F9EE3AFA7D087C0012799F53E8EF901871
:105D1A007FE02408F0C39438401490167EE4F09093
:105D2A001550E0243DF08006127D0253E8EFE5E8C5
:105D3A0020E303025E20901704E0640160089018D3
:105D4A00C1E064017030E5ED30E61F901709E0B458
:105D5A00010F901704E4F09018C1F0901709F08031
:105D6A00091279E69017097401F063ED8053E8F798
:105D7A0075EAB0025E20E5ED30E61F1279E6900181
:105D8A006AEFF053E8F7E07003025E2012701AEF30
:105D9A006003025E20127B5D807CE5ED540F606437
:105DAA00901839E0C39440505BE5ED540F900168B8
:105DBA00F0E4FE900168E0FFEEC39F50149018399A
:105DCA00E02E243CF582E43418F583E5EFF00E80EA
:105DDA00E263ED8053E8F7125104900168E0FF9006
:105DEA001839E02FF0C39440402C127A2B75EAB090
:105DFA0090187CE0B4011F9018C17401F090187CCF
:105E0A00E4F0801290170AE0B40105E4F012701A67
:105E1A0063ED8053E8F7E5E830E20353E8FBE5E891
:105E2A0030E00353E8FEE5E830E70353E87FE5E8AE
:095E3A0030E50653E8DF1274CADA
:105E4300D007D006D005D004D003D002D001D000B3
:0B5E5300D0D0D082D083D0F0D0E0325D
:08753F00900101EEF0A3EFF052
:10754700E4FFF990955574AAF0909AAA7455F090B3
:10755700955574A0F0900101E0FAA3E0F5828A83C3
:10756700EDF05480FD900101E0FAA3E0F5828A83F3
:10757700E0FE5420FCEE5480FEB505047F01800632
:10758700ECB420027901EF7003E960D9E964017076
:1075970019900101E0FAA3E0F5828A83E05480B5EF
:0A75A70005027F0190955574F0F085
:0175B10022B7
:1077B200E4FDFC90955574AAF0909AAA7455F09045
:1077C20095557480F074AAF0909AAA7455F08F823D
:1077D2008E837430F08F828E83E0FB5420F9EB5459
:1077E20080FBB480047D018006E9B420027C01EDB7
:1077F2007003EC60E0ECB401128F828E83E054805F
:0D780200B480027D0190955574F0F0AF0543
:01780F002256
:10200F000223C4E86480F8E933E83360110460F018
:10201F00ED33EC337009E8FCE9FDEAFEEBFF220437
:10202F0060DED3EB9FEA9EE99DE8C2E78CF0C2F732
:10203F0095F0400CE8CCF8E9CDF9EACEFAEBCFFBFE
:10204F0012238F85D0F05804700320D5B3E80470A5
:10205F00075002B2D50223CE92D5EC0460F7E4CC40
:10206F00C0E0C398F8603B94186008400DD0E0FBC7
:10207F000223A6E4FBFAC9FC8028E830E406E4C991
:10208F00FBE4CAFCE830E305E4C9CACBFCE854071B
:10209F006010F8C3E913F9EA13FAEB13FBEC13FC26
:1020AF00D8F130F52FC3E49CFCEF9BFFEE9AFEEDC9
:1020BF0099FDD0E0FBEF4E4D4C701222DB03022353
:1020CF00CBEC2CFCEF33FFEE33FEED33FDED30E7C1
:1020DF00EB0223A6EF2BFFEE3AFEED39FDD0E0FB2E
:1020EF0050130BBB00030223CEED13FDEE13FEEFD7
:0820FF0013FFEC13FC0223A601
:10210700EC4D6011E8497017ED33EC3304600DE4D2
:10211700FCFFFEFD22E933E8330470F80223C41202
:10212700238F58046009E4CC248150062850090203
:1021370023CE2840030223CBC0E0EB4A7044B9808A
:1021470006D0E0FB0223BAEF4E701CBD8008EBFF00
:10215700EAFEE9FD80EBE98DF0A4FEE5F00221F04F
:10216700E9CDF9EAFEEBFFEF89F0A4FCE5F0CE89B3
:10217700F0A42EFFE435F0CD89F0A42DFEE435F070
:102187008067EF4E7005BD80D780C3EF8BF0A4AC9E
:10219700F0EE8BF0A42CFCE435F0F8EF8AF0A42CD9
:1021A700E5F038FCE433CB8DF0A42CFCE5F03BF8EC
:1021B700EE8AF0A42CFCE5F038F8E433CF89F0A4DC
:1021C7002CFCE5F038CF3400CE89F0A42FFFE5F0E2
:1021D7003EFEE433C98DF0A42EFEE5F039CD8AF03A
:1021E700A42FFFE5F03EFEE43DFD33D0E0FB5007B2
:1021F7000BBB000F0223CEEC2CFCEF33FFEE33FEBC
:06220700ED33FD0223A6E9
:10220D000223CEEC5D046005E8590470030223C47B
:10221D0012238F580460F6EC4860F2EC7004FDFE5A
:10222D00FF22C860DB2481C85009C39860025006A4
:10223D000223CB9850CAF582E9294B4A7005AB822F
:10224D000223BA75F0007C1A7880C3EF9BEE9AEDED
:10225D0099400DC3EF9BFFEE9AFEED99FDE842F01C
:10226D00DC23ACF0D0E0FFD0E0FED0E0FDAB82206F
:10227D00E7101BEB60BAEC2CFCEF33FFEE33FEEDF9
:10228D0033FD0223A6E803F830E705C0F075F00032
:10229D00EF2FFFEE33FEED33FD40B830E7C280AADD
:1022AD0074F8CC6480CCC86480C8F582046043C3E4
:1022BD00EB9FF5F0EA9E42F0E99D42F0E89C45F077
:1022CD0060305018E5825FFFE582F42B5582FB509C
:1022DD00210ABA001D09B90019088016E5825BFBB9
:1022ED00E582F42F5582FF50090EBE00050DBD008D
:1022FD00010CC3EB9FF5F0EA9E42F0E99D42F0E838
:0D230D009C45F06007CC4820E701B3EC22AE
:10231A0075F020800E75F010800575F0087D007E3E
:10232A00007F003392D530D5031228E1EC334010F8
:10233A00EF33FFEE33FEED33FDEC33FCD5F0ED2247
:0E234A00E5F0247EA2D513CC92E7CDCEFF2283
:10235800EDD2E7CD33EC3392D524814006E4FFFE7D
:10236800FDFC22FCE4CFCECDCC24E0501174FF80DC
:10237800EDC3CC13CCCD13CDCE13CECF13CF047079
:07238800F030D5DE0228E170
:103E9100E516243BF582E43401F583E00516229012
:103EA100013830070390013BE475F00112295C02EF
:103EB10026812000E97F2ED2008018EF540F249034
:103EC100D43440D4FF30040BEF24BFB41A005003A4
:103ED1002461FFE51760021517051AE51A7002053E
:103EE1001930070E900138E475F00112295CEF02D8
:103EF10026C7027CB57403D2078003E4C207F51616
:103F0100900138122973E4F517F519F51AE51760D0
:103F1100077F20123ED480F57518FFC201C200C28E
:103F210002C203C205C206C208123EA0FF700D30D4
:103F310007057F00123EE5AF1AAE1922B4255FC214
:103F4100D5C204123EA0FF24D0B40A00501A75F065
:103F51000A781730D50508B6FF0106C6A426F62053
:103F6100D5047002D20380D924CFB41A00EF5004D3
:103F7100C2E5D2040241D7D20180C6D20080C0D2AC
:103F81000280BCD2D580BAD20580B47F20123ED443
:103F91002002077401B5170040F1123E91FF123E55
:103FA100D4023F0ED208D2068095123E91FB123EFA
:103FB10091FA123E91F94A4B700679D57A427BFF0C
:103FC10020022EE517602A7E008E8275830012265C
:103FD1009A60060EEE651870F0C2D5EBC0E0EAC03B
:103FE100E0E9C0E0EE124238D0E0F9D0E0FAD0E0EA
:103FF100FB122681FF60AAEBC0E0EAC0E0E9C0E065
:10400100123ED4D0E02401F9D0E03400FAD0E0FB34
:10401100E5180460DCD518D98087D20280A212424B
:104021001A60F7E5187001041223D9A918600DE58B
:1040310018600914F5181242C2EF60F3EA30E70282
:10404100F404C3995079EAF425180430E701E40433
:10405100F518800D12421A60C1EA051825181223BD
:10406100D9EA900167F030E701E4251804D5180476
:1040710020050114124238E4C0E01242C2900167E7
:10408100E0601320E70714F0123EBC802204F0D058
:10409100E014C0E07F00123EBCE5186007123EB399
:1040A1001518800B300503123EB3D0E0023F0ED04D
:1040B100E00480C412421A609EE518041223D990CC
:1040C1000167EAF0E51820050260010424041242A8
:0140D10038B6
:1040D20074FF04C0E01242C2123EBCE51820050281
:1040E2006003123EB3D0E0B518E87F45123EC69099
:1040F2000167E07F2B30E7047F2DF404C0E0123E1D
:10410200D4D0E075F00A84C0F0123EBDD0E0123E79
:10411200BD023F0E791080027908C206C2088008EB
:10412200D2D5790A8004790AC2D5E518047002F55D
:1041320018E4FAFDFEFF123E91FC7B0820011312E7
:104142003E91FD7B1030000A123E91FE123E91FF1D
:104152007B20EC3382D592D55013C3E43000069F06
:10416200FFE49EFEE42001039DFDE49CFCE4CBF809
:10417200C201EC700CCFCECDCCE824F8F870F380FD
:1041820017C3EF33FFEE33FEED33FDEC33FCEB33BD
:10419200FB994002FB0FD8E9EB300105F8D0E0C4EF
:1041A20048B201C0E00AEC4D4E4F78207B0070C24D
:1041B200EAB5180040BCC0E012423AD0F0D0E0208C
:1041C2000104C4C0E0C4B201C0F0123EBDD0F0D5BB
:1041D200F0EB023F0E12297C3FAB534116583F7C55
:1041E2004C3F7842411A4F4122444122493F914378
:1041F20041285540554640B545401F4742F5503F7E
:10420200802D3F842E3FA72B3F88233FA52042DEEF
:104212002A3F404800003F9FE518B4FF0375180687
:10422200123E91FC123E91FD123E91FE123E91FF12
:10423200900160022416790AA2D5200314300509E0
:10424200B910020404B9080104A2D52006025001E3
:10425200042002689202B517005034C0E07F20307B
:1042620003197F30A20272067205500F124291C2E8
:1042720002C206C205C2087F30800F300503E9C0C2
:10428200E0123ED4300503D0E0F9D0E0B517CC30CF
:1042920005177F30B9100C123ED47F583004077FC7
:1042A200788003B90803123ED43002057F2D023E06
:1042B200D47F202008F87F2B2006F322920280CFA1
:1042C2007F00B40700500B2460F582E43401F583CB
:1042D200E0FF22286E756C6C2900D201123E9130EB
:1042E20001F8C201781730D50108F6023F402D507F
:1042F200434958123E912403B405004001E4904220
:10430200F093123EC5743A123EC5D20375170402E9
:02431200411652
:10238F00E9D2E7C933E833F892D5EDD2E7CD33EC94
:07239F0033FC5002B2D5220D
:1023A600EC30E7100FBF000C0EBE00080DBD000498
:1023B6000BEB6014A2D5EB13FCED92E7FD2274FF44
:1023C600FCFDFEFF22E480F8A2D574FF13FC7D809D
:0323D600E480EFB1
:1023D900F920E73624F950037907E4F42402FBE5F0
:1023E90082158270021583DBF6E024FB501BE9603D
:1023F90014E4F0E582158270021583E004F0B40A52
:0D24090008E4F0D9EE7401F00A22C2D522D9
:10241600ED33EC3392D5FA602AB4FF33EDC2E77B95
:10242600FF60067A24793BE4227A24794420D50495
:102436007A24793F224E614E002B494E46002D49A3
:102446004E4600E47A08F0A3DAFC7B00740722C04B
:1024560083C082ECC0E0EDC0E0EEC0E0EFC0E0EA91
:1024660075F010A4CAABF075F04DA42BFBE435F063
:10247600FCEA2410FAEB34C5FBEC34D9FCEDC2E7D8
:10248600FF75F056A4F42411C5F0F434C58FF0A4FA
:102496002AE5F03BE43CF020E71412254BD0E0FFA0
:1024A600D0E0FED0E0FDD0E0FC1222108014F4044F
:1024B60012254BD0E0FFD0E0FED0E0FDD0E0FC12CC
:1024C6002107D082D083E0FAEDD2E7CD33EC332476
:1024D60082FBE4C3CF33CFCE33CECD33CD33DBF364
:1024E6007B0775F00A846004F0A31B0AE5F0F0A3ED
:1024F6008FF0740AA4FFACF08EF0740AA42CFEAC24
:10250600F050010C8DF0740AA42CFDE435F0F0A314
:05251600DBDE7407226A
:10251B003F8000004120000042C80000447A0000C8
:10252B00461C400047C35000497424004B1896804A
:10253B004CBEBC205A0E1BCA6753C21C749DC5AE41
:10254B00FB60065407601C2323122579EB5438607B
:10255B0009122565122574122107ECF8EDF9EEFA34
:10256B00EFCB22EB12257480F1543803241C9025F9
:10257B001BFE93FC0EEE93FD0EEE930ECE93FF22FD
:1072CE0002734EE493A3F8E493A34003F68001F215
:1072DE0008DFF48029E493A3F85407240CC8C333C1
:1072EE00C4540F4420C8834004F456800146F6DF90
:1072FE00E4800B0102040810204080903936E47EB1
:10730E00019360BCA3FF543F30E509541FFEE49384
:10731E00A360010ECF54C025E060A840B8E493A34B
:10732E00FAE493A3F8E493A3C8C582C8CAC583CA76
:10733E00F0A3C8C582C8CAC583CADFE9DEE780BE2E
:013E90000031
:10258B00E709F608DFFA8046E709F208DFFA803E32
:10259B0088828C83E709F0A3DFFA8032E309F6081F
:1025AB00DFFA8078E309F208DFFA807088828C8387
:1025BB00E309F0A3DFFA806489828A83E0A3F6083B
:1025CB00DFFA805889828A83E0A3F208DFFA804C15
:1025DB0080D280FA80C680D4806980F280338010EC
:1025EB0080A680EA809A80A880DA80E280CA803355
:1025FB0089828A83ECFAE493A3C8C582C8CCC583CD
:10260B00CCF0A3C8C582C8CCC583CCDFE9DEE7809C
:10261B000D89828A83E493A3F608DFF9ECFAA9F01B
:10262B00EDFB2289828A83ECFAE0A3C8C582C8CC71
:10263B00C583CCF0A3C8C582C8CCC583CCDFEADE8A
:10264B00E880DB89828A83E493A3F208DFF980CCEC
:10265B0088F0EF60010E4E60C388F0ED2402B404E5
:10266B000050B9F582EB2402B4040050AF2323458C
:06267B0082239025DB73B1
:10268100BB010689828A83E0225002E722BBFE0257
:09269100E32289828A83E493228A
:10269A00BB010CE58229F582E5833AF583E02250F5
:1026AA0006E92582F8E622BBFE06E92582F8E2223F
:0D26BA00E58229F582E5833AF583E4932259
:1026C700BB010689828A83F0225002F722BBFE01F2
:0226D700F322EC
:1026D900EF8DF0A4A8F0CF8CF0A428CE8DF0A42E15
:0226E900FE22CF
:1026EB00BC000BBE0029EF8DF084FFADF022E4CCD3
:1026FB00F875F008EF2FFFEE33FEEC33FCEE9DEC9C
:10270B00984005FCEE9DFE0FD5F0E9E4CEFD22EDE1
:10271B00F8F5F0EE8420D21CFEADF075F008EF2F2B
:10272B00FFED33FD4007985006D5F0F222C398FD1C
:05273B000FD5F0EA22B9
:10274000C2D5EC30E709B2D5E4C39DFDE49CFCEEB4
:1027500030E715B2D5E4C39FFFE49EFE1226EBC31B
:10276000E49DFDE49CFC80031226EB30D507C3E416
:062770009FFFE49EFE2223
:10277600A3F8E0C5F025F0F0E58215827002158316
:06278600E0C838F0E82273
:10278C00BB0110E58229F582E5833AF583E0F5F08B
:10279C00A3E0225009E92582F886F008E622BBFE68
:1027AC000AE92582F8E2F5F008E222E5832AF583AE
:0827BC00E993F5F0A3E9932273
:1027C400E88FF0A4CC8BF0A42CFCE98EF0A42CFCB4
:1027D4008AF0EDA42CFCEA8EF0A4CDA8F08BF0A432
:1027E4002DCC3825F0FDE98FF0A42CCD35F0FCEB91
:1027F4008EF0A4FEA9F0EB8FF0A4CFC5F02ECD3956
:0F280400FEE43CFCEAA42DCE35F0FDE43CFC22C2
:1028130075F008758200EF2FFFEE33FECD33CDCC7C
:1028230033CCC58233C5829BED9AEC99E5829840FF
:102833000CF582EE9BFEED9AFDEC99FC0FD5F0D6DC
:10284300E4CEFBE4CDFAE4CCF9A88222B800C1B906
:102853000059BA002DEC8BF084CFCECDFCE5F0CB44
:10286300F97818EF2FFFEE33FEED33FDEC33FCEB7D
:1028730033FB10D703994004EB99FB0FD8E5E4F938
:10288300FA227818EF2FFFEE33FEED33FDEC33FC25
:10289300C933C910D7059BE99A4007EC9BFCE99A19
:1028A300F90FD8E0E4C9FAE4CCFB2275F010EF2F5E
:1028B300FFEE33FEED33FDCC33CCC833C810D7075E
:1028C3009BEC9AE899400AED9BFDEC9AFCE899F899
:0E28D3000FD5F0DAE4CDFBE4CCFAE4C8F9222C
:0E28E100C3E49FFFE49EFEE49DFDE49CFC2208
:1028EF00EB9FF5F0EA9E42F0E99D42F0E89C45F03F
:0128FF0022B6
:10290000E8600FECC313FCED13FDEE13FEEF13FFB5
:03291000D8F122D9
:0C291300ECF0A3EDF0A3EEF0A3EFF02237
:10291F00A8828583F0D083D08212293612293612ED
:10292F002936122936E473E493A3C583C5F0C58312
:10293F00C8C582C8F0A3C583C5F0C583C8C582C802
:01294F002265
:0C295000A42582F582E5F03583F5832292
:10295C00F8E0FBA3A3E0F925F0F0E5821582700204
:07296C001583E0FA38F022A8
:09297300EBF0A3EAF0A3E9F02265
:10297C00D083D082F8E4937012740193700DA3A3EA
:10298C0093F8740193F5828883E4737402936860FE
:06299C00EFA3A3A380DFFE
:107CB500EFB40A07740D127CC0740A309811A899A4
:107CC500B8130CC2983098FDA899C298B811F6302F
:077CD50099FDC299F5992207
:107623009000FBEBF0A3EAF0A3E9F0900101EBF08B
:10763300A3EAF0A3E9F09000FBE0FBA3E475F001FB
:10764300122776A9F0FA12268170EB9000FC74FFE2
:10765300F5F0122AB79000FEE0FBA3E475F00112E7
:107663002776A9F0FA122681FF9000FBE0FBA3E442
:1076730075F001122776A9F0FAEF1226C770D6909B
:0B7683000101E0FBA3E0FAA3E0F92204
:1029A200E709F60870FA8046E709F20870FA803EF5
:1029B20088828C83E709F0A370FA807EE309F60827
:1029C20070FA8076E309F20870FA806E88828C834E
:1029D200E309F0A370FA806289828A83E0A3F60891
:1029E20070FA805689828A83E0A3F20870FA804ADC
:1029F20080D280FA80C680D4806580F280318010D7
:102A020080A680EA809A80A880DA80E280CA80313B
:102A120089828A83ECFAE493A3C8C582C8CCC583B1
:102A2200CCF0A3C8C582C8CCC583CC70E9800D891F
:102A3200828A83E493A3F60870F9ECFAA9F0EDFB1D
:102A42002289828A83ECFAE0A3C8C582C8CCC583F6
:102A5200CCF0A3C8C582C8CCC583CC70EA80DD891E
:102A6200828A83E493A3F20870F980CE88F0ED2481
:102A720002B4040050C4F582EB2402B4040050BA3C
:092A820023234582239029F273FD
:102A8B00EF4E6012EF60010EEDBB010B89828A8362
:102A9B00F0A3DFFCDEFA2289F05007F709DFFCA96F
:0C2AAB00F022BBFEFCF309DFFCA9F022C6
:102AB700C5F0F8A3E028F0C5F0F8E58215827002AA
:062AC7001583E038F02247
:00000001FF
